:020000040000FA
:0408000098EF0BF072
:1008100003B275EF05F0F2B493EF05F09EB09BEFD5
:1008200005F09EB2A3EF05F0F2A81AEF04F0F2B2C1
:1008300023EF04F0F2B01FEF04F047EF0BF0F29655
:10084000F29047EF0BF0CD90F2929EA02DEF04F0C6
:100850000101533F2DEF04F0542BB2C1B6F1B3C1E7
:10086000B7F1B4C1B8F1B5C1B9F1AEC1B2F1AFC120
:10087000B3F1B0C1B4F1B1C1B5F1AAC1AEF1ABC130
:10088000AFF1ACC1B0F1ADC1B1F1A6C1AAF1A7C140
:10089000ABF1A8C1ACF1A9C1ADF1A2C1A6F1A3C150
:1008A000A7F1A4C1A8F1A5C1A9F19EC1A2F19FC160
:1008B000A3F1A0C1A4F1A1C1A5F19AC19EF19BC170
:1008C0009FF19CC1A0F19DC1A1F1CECF9AF1CFCFF4
:1008D0009BF153C19CF154C19DF1CF6ACE6A0101D5
:1008E000536B546B9E90CD800FBC0F8E0FBA7CEF74
:1008F00004F00F8A47EF0BF013880F8C0FBEB9EF8F
:1009000004F09AC19EF19BC19FF19CC1A0F19DC1D1
:10091000A1F19EC1A2F19FC1A3F1A0C1A4F1A1C107
:10092000A5F1A2C1A6F1A3C1A7F1A4C1A8F1A5C1D7
:10093000A9F1A6C1AAF1A7C1ABF1A8C1ACF1A9C1A7
:10094000ADF1AAC1AEF1ABC1AFF1ACC1B0F1ADC177
:10095000B1F1AEC1B2F1AFC1B3F1B0C1B4F1B1C147
:10096000B5F1B2C1B6F1B3C1B7F1B4C1B8F1B5C117
:10097000B9F101015E6B5F6B606B616B9A515E2731
:100980009B515F239C5160239D5161239E515E27A3
:100990009F515F23A0516023A1516123A2515E2783
:1009A000A3515F23A4516023A5516123A6515E2763
:1009B000A7515F23A8516023A9516123AA515E2743
:1009C000AB515F23AC516023AD516123AE515E2723
:1009D000AF515F23B0516023B1516123B2515E2703
:1009E000B3515F23B4516023B5516123B6515E27E3
:1009F000B7515F23B8516023B9516123D8900101E9
:100A0000613360335F335E33D8900101613360330B
:100A10005F335E33D8900101613360335F335E33FF
:100A200000C10CF101C10DF102C10EF103C10FF1C2
:100A300004C110F105C111F106C112F107C113F192
:100A400008C114F109C115F10AC116F10BC117F162
:100A500034C135F111B838EF05F00101620E046FB1
:100A6000010E056F000E066F000E076F41EF05F0D7
:100A70000101A70E046F020E056F000E066F000E37
:100A8000076F5EC100F15FC101F160C102F161C198
:100A900003F100EC30F003BF04D01CBE02D01CA058
:100AA000108C11A059EF05F010BA59EF05F00F8026
:100AB000108A0CC100F10DC101F10EC102F10FC18C
:100AC00003F110C104F111C105F112C106F113C106
:100AD00007F114C108F115C109F116C10AF117C1D6
:100AE0000BF135C134F147EF0BF00392ABB2AB9889
:100AF000AB88030103EE00F080517F0BE92604C0B0
:100B0000EFFF802B8151805D700BD8A48B82000099
:100B10008051815D700BD8A48B9281518019D8B41B
:100B2000079047EF0BF0F2940101453F47EF0BF0C0
:100B3000462B47EF0BF09E900101533F47EF0BF020
:100B4000542B47EF0BF09E9211B843EF08F00400CE
:100B500066A1ABEF05F08BB4B5EF05F010ACB5EFC7
:100B600005F08B84109CB6EF05F08B94077C07ACE6
:100B7000D1EF05F0C274C2B4CBEF05F0C3CFB7F527
:100B8000C4CFB8F50501D890B833B733D890B8338F
:100B9000B733D2EF05F0C3CF55F1C4CF56F1D2EF42
:100BA00005F0C28207B444EF06F047C14BF148C1DB
:100BB0004CF149C14DF14AC14EF15EC162F15FC1D4
:100BC00063F160C164F161C165F113A8EAEF05F05A
:100BD000138C13989AC1BAF19BC1BBF19CC1BCF1B3
:100BE0009DC1BDF19EC1BEF19FC1BFF1A0C1C0F1C9
:100BF000A1C1C1F1A2C1C2F1A3C1C3F1A4C1C4F199
:100C0000A5C1C5F1A6C1C6F1A7C1C7F1A8C1C8F168
:100C1000A9C1C9F1AAC1CAF1ABC1CBF1ACC1CCF138
:100C2000ADC1CDF1AEC1CEF1AFC1CFF1B0C1D0F108
:100C3000B1C1D1F1B2C1D2F1B3C1D3F1B4C1D4F1D8
:100C4000B5C1D5F1B6C1D6F1B7C1D7F1B8C1D8F1A8
:100C5000B9C1D9F1B7C5B9F5B8C5BAF5B9C5BBF5CC
:100C6000BAC5BCF5010155515B2756515C23E86AB2
:100C70005D230E2E44EF06F05CC157F15DC158F1C3
:100C80005B6B5C6B5D6B078E0201002F47EF0BF017
:100C90003C0E006F1D50E00BE00AE86612881BBE98
:100CA00002D01BB4108E00C10CF101C10DF102C1C4
:100CB0000EF103C10FF104C110F105C111F106C11C
:100CC00012F107C113F108C114F109C115F10AC1EC
:100CD00016F10BC117F134C135F181AAACEF06F062
:100CE00015A4F7EF06F005012F51000AD8B43AEF2A
:100CF00007F005012F51010AD8B4B6EF06F005013F
:100D00002F51020AD8B4F7EF06F005012F51030A5C
:100D1000D8B4F7EF06F005012F51040AD8B4F7EF65
:100D200006F005012F51050AD8B4F7EF06F00501CA
:100D30002F51060AD8B4F7EF06F005012F51070A24
:100D4000D8B4F7EF06F005012F51320AD8B4B4EF4A
:100D500006F02F6B3AEF07F000011650030AD8B4E3
:100D6000F7EF06F03AEF07F03AEF07F005015767A3
:100D7000C1EF06F05867C1EF06F05967C1EF06F002
:100D80005A67C5EF06F03AEF07F05BC500F15CC5A6
:100D900001F15DC502F15EC503F10101010E046FB1
:100DA000000E056F000E066F000E076F00EC30F0AE
:100DB00000C15BF501C15CF502C15DF503C15EF5E3
:100DC00001010067EBEF06F00167EBEF06F0026749
:100DD000EBEF06F003673AEF07F057C55BF558C530
:100DE0005CF559C55DF55AC55EF524EF07F00FBEF9
:100DF0000CEF07F010A011EF07F00101476708EFB3
:100E000007F0486708EF07F0496708EF07F04A67FF
:100E10000CEF07F011EF07F007AE11EF07F024EF2A
:100E200007F00501312F3AEF07F03C0E316F302FFC
:100E30003AEF07F00101000E626FE00E636FA50E3E
:100E4000646F010E656F138800011650000AD8B454
:100E500032EF07F000011650030AD8B437EF07F05D
:100E60003AEF07F00001010E166E3AEF07F00001AD
:100E7000040E166E0501666B37B740EF07F066810A
:100E80000CC100F10DC101F10EC102F10FC103F15E
:100E900010C104F111C105F112C106F113C107F12E
:100EA00014C108F115C109F116C10AF117C10BF1FE
:100EB00035C134F100C10CF101C10DF102C10EF1D7
:100EC00003C10FF104C110F105C111F106C112F106
:100ED00007C113F108C114F109C115F10AC116F1D6
:100EE0000BC117F134C135F101018E677FEF07F0B7
:100EF0008F677FEF07F090677FEF07F0916783EFD1
:100F000007F0B4EF07F092C100F193C101F194C171
:100F100002F195C103F10101010E046F000E056F8E
:100F2000000E066F000E076F00EC30F000C192F16A
:100F300001C193F102C194F103C195F10101006770
:100F4000A9EF07F00167A9EF07F00267A9EF07F023
:100F50000367B4EF07F08EC192F18FC193F190C196
:100F600094F191C195F10F80D57ED5BE6ED0D6CFCC
:100F700047F1D7CF48F145C149F1E86AE8CF4AF1D6
:100F8000138A1CBE02D01CA0108C109047C100F127
:100F900048C101F149C102F14AC103F101010A0E40
:100FA000046F000E056F000E066F000E076F00EC59
:100FB00030F003AF1080010154A7EBEF07F00F9A58
:100FC0000F9C0F9E0101000E5E6F600E5F6F3D0E65
:100FD000606F080E616F010147BFFBEF07F04867C4
:100FE000FBEF07F04967FBEF07F04A67FBEF07F0FD
:100FF000F28820EF08F0F2985E6B5F6B606B616BBC
:101000009A6B9B6B9C6B9D6B9E6B9F6BA06BA16B9C
:10101000A26BA36BA46BA56BA66BA76BA86BA96B4C
:10102000AA6BAB6BAC6BAD6BAE6BAF6BB06BB16BFC
:10103000B26BB36BB46BB56BB66BB76BB86BB96BAC
:10104000D76AD66A0101456B466B0CC100F10DC130
:1010500001F10EC102F10FC103F110C104F111C180
:1010600005F112C106F113C107F114C108F115C150
:1010700009F116C10AF117C10BF135C134F147EF7F
:101080000BF047EF0BF00201002FABEF0AF0D59EFB
:10109000D6CF47F1D7CF48F145C149F1E86AE8CF4B
:1010A0004AF1138AD76AD66A0101456B466BD58E21
:1010B0001D50E00BE00AE86612881BBE02D01BB48C
:1010C000108E1AAE1F8C00C10CF101C10DF102C1CE
:1010D0000EF103C10FF104C110F105C111F106C1F8
:1010E00012F107C113F108C114F109C115F10AC1C8
:1010F00016F10BC117F134C135F10FA0109A11B8D8
:101100008DEF08F00101620E046F010E056F000EF5
:10111000066F000E076F96EF08F00101A70E046F2F
:10112000020E056F000E066F000E076F47C100F13B
:1011300048C101F149C102F14AC103F100EC30F0AC
:1011400003BFA9EF08F01CBE02D01CA0108C11B088
:101150000F800CC100F10DC101F10EC102F10FC1F0
:1011600003F110C104F111C105F112C106F113C15F
:1011700007F114C108F115C109F116C10AF117C12F
:101180000BF135C134F102013C0E006F00C10CF1CE
:1011900001C10DF102C10EF103C10FF104C110F143
:1011A00005C111F106C112F107C113F108C114F113
:1011B00009C115F10AC116F10BC117F134C135F19E
:1011C00081BAE6EF08F015B225EF09F015A025EF7A
:1011D00009F015A470EF09F005012F51000AD8B4E9
:1011E000B3EF09F005012F51010AD8B42FEF09F030
:1011F00005012F51020AD8B470EF09F005012F51F3
:10120000030AD8B470EF09F005012F51040AD8B4CD
:1012100070EF09F005012F51050AD8B470EF09F0FD
:1012200005012F51060AD8B470EF09F005012F51BE
:10123000070AD8B470EF09F005012F51320AD8B46B
:101240002DEF09F02F6BB3EF09F000011650030AE0
:10125000D8B470EF09F0B3EF09F0B3EF09F005016E
:1012600057673AEF09F058673AEF09F059673AEFD4
:1012700009F05A673EEF09F0B3EF09F05BC500F1E2
:101280005CC501F15DC502F15EC503F10101010E0E
:10129000046F000E056F000E066F000E076F00EC66
:1012A00030F000C15BF501C15CF502C15DF503C121
:1012B0005EF50101006764EF09F0016764EF09F072
:1012C000026764EF09F00367B3EF09F057C55BF5F8
:1012D00058C55CF559C55DF55AC55EF59DEF09F039
:1012E0000FBE85EF09F010A08AEF09F001014767F2
:1012F00081EF09F0486781EF09F0496781EF09F054
:101300004A6785EF09F08AEF09F007AE8AEF09F026
:101310009DEF09F00501312FB3EF09F03C0E316F5D
:10132000302FB3EF09F00101000E626FE00E636F22
:10133000A50E646F010E656F138800011650000A38
:10134000D8B4ABEF09F000011650030AD8B4B0EFDF
:1013500009F0B3EF09F00001010E166EB3EF09F0CA
:101360000001040E166E0501666B37B7B9EF09F080
:1013700066810CC100F10DC101F10EC102F10FC176
:1013800003F110C104F111C105F112C106F113C13D
:1013900007F114C108F115C109F116C10AF117C10D
:1013A0000BF135C134F100C10CF101C10DF102C1E5
:1013B0000EF103C10FF104C110F105C111F106C115
:1013C00012F107C113F108C114F109C115F10AC1E5
:1013D00016F10BC117F134C135F101018E67F8EF39
:1013E00009F08F67F8EF09F09067F8EF09F091675F
:1013F000FCEF09F02DEF0AF092C100F193C101F169
:1014000094C102F195C103F10101010E046F000EB8
:10141000056F000E066F000E076F00EC30F000C184
:1014200092F101C193F102C194F103C195F101015F
:10143000006722EF0AF0016722EF0AF0026722EF4D
:101440000AF003672DEF0AF08EC192F18FC193F17C
:1014500090C194F191C195F10F80109047C100F1B6
:1014600048C101F149C102F14AC103F101010A0E6B
:10147000046F000E056F000E066F000E076F00EC84
:1014800030F003AF1080010154A753EF0AF00F9A18
:101490000F9C0F9E0101000E5E6F600E5F6F3D0E90
:1014A000606F080E616F47C100F148C101F149C189
:1014B00002F14AC103F10101140E046F050E056F1C
:1014C000000E066F000E076F00EC30F003AF6CEFFC
:1014D0000AF0F28891EF0AF0F2985E6B5F6B606B36
:1014E000616B9A6B9B6B9C6B9D6B9E6B9F6BA06BF8
:1014F000A16BA26BA36BA46BA56BA66BA76BA86B70
:10150000A96BAA6BAB6BAC6BAD6BAE6BAF6BB06B1F
:10151000B16BB26BB36BB46BB56BB66BB76BB86BCF
:10152000B96B0CC100F10DC101F10EC102F10FC187
:1015300003F110C104F111C105F112C106F113C18B
:1015400007F114C108F115C109F116C10AF117C15B
:101550000BF135C134F104008BB4B6EF0AF010ACD6
:10156000B6EF0AF08B84109CB7EF0AF08B94077CDF
:1015700007ACD2EF0AF0C274C2B4CCEF0AF0C3CF0A
:10158000B7F5C4CFB8F50501D890B833B733D890C4
:10159000B833B733D3EF0AF0C3CF55F1C4CF56F108
:1015A000D3EF0AF0C28207B445EF0BF047C14BF10D
:1015B00048C14CF149C14DF14AC14EF15EC162F1E1
:1015C0005FC163F160C164F161C165F113A8EBEF24
:1015D0000AF0138C13989AC1BAF19BC1BBF19CC15C
:1015E000BCF19DC1BDF19EC1BEF19FC1BFF1A0C1C3
:1015F000C0F1A1C1C1F1A2C1C2F1A3C1C3F1A4C193
:10160000C4F1A5C1C5F1A6C1C6F1A7C1C7F1A8C162
:10161000C8F1A9C1C9F1AAC1CAF1ABC1CBF1ACC132
:10162000CCF1ADC1CDF1AEC1CEF1AFC1CFF1B0C102
:10163000D0F1B1C1D1F1B2C1D2F1B3C1D3F1B4C1D2
:10164000D4F1B5C1D5F1B6C1D6F1B7C1D7F1B8C1A2
:10165000D8F1B9C1D9F1B7C5B9F5B8C5BAF5B9C5A9
:10166000BBF5BAC5BCF5010155515B2756515C234A
:10167000E86A5D230E2E45EF0BF05CC157F15DC1AA
:1016800058F15B6B5C6B5D6B078E47EF0BF002C034
:10169000E0FF005001C0D8FF1000A6B24DEF0BF0E4
:1016A0000CC0A9FF0BC0A8FFA69EA69CA684F29E14
:1016B000550EA76EAA0EA76EA682F28EA694A6B2AB
:1016C0005FEF0BF00C2A1200A96EA69EA69CA680C6
:1016D000A8500C2A120004012C0E826F96EC0EF01A
:1016E00015EC31F00C5064EC0BF0E8CF00F10C502D
:1016F00064EC0BF0E8CF01F101AF84EF0BF00101D6
:10170000FF0E026FFF0E036F9EEC30F0296790EF23
:101710000BF00401200E826F96EC0EF095EF0BF0AB
:1017200004012D0E826F96EC0EF0A8EC2EF0120044
:1017300015941596076A0F6A106A116A126A136A7D
:10174000166A0F010D0EC16E860EC06E030EC26EBC
:101750000F01680E896E130E926E080E8A6EF30EDC
:10176000936E8B6A900E946EC80E64EC0BF0E8CF0B
:10177000E8FF1098E8A0108810A805D00E0E256E7E
:101780008E0E266E04D00F0E256E8F0E266EADECDB
:1017900031F0F8EC32F0F18EF19EFC0E64EC0BF0BF
:1017A000E8CF0BF00BA011800BA211820BA41184C7
:1017B0000BA81188C90E64EC0BF0E8CF1AF0CA0E22
:1017C00064EC0BF0E8CF1BF0CB0E64EC0BF0E8CF31
:1017D0001CF0CC0E64EC0BF0E8CF1DF0FB0E64ECBB
:1017E0000BF0E8CF37F0CE0E64EC0BF0E8CF14F03E
:1017F000CD0E64EC0BF0E8CF36F01F6A206A0E6A5B
:1018000001015B6B5C6B5D6B576B586BF29A01016E
:10181000476B486B496B4A6B4B6B4C6B4D6B4E6B1C
:101820004F6B506B516B526B456B466BD76AD66AE8
:101830000F01280ED56EF28A9D90B00ECD6E01017B
:101840005E6B5F6B606B616B626B636B646B656B34
:10185000666B676B686B696B536B546BCF6ACE6A50
:101860000F9A0F9C0F9E9D80760ECA6E9D8202017C
:101870003C0E006FCC6A160E64EC0BF0E8CF00F162
:10188000170E64EC0BF0E8CF01F1180E64EC0BF0CE
:10189000E8CF02F1190E64EC0BF0E8CF03F101017F
:1018A00003AF6DEF0CF015EC31F0160E0C6E00C1AD
:1018B0000BF04DEC0BF0170E0C6E01C10BF04DEC64
:1018C0000BF0180E0C6E02C10BF04DEC0BF0190E64
:1018D0000C6E03C10BF04DEC0BF000C18EF101C199
:1018E0008FF102C190F103C191F100C192F101C1E8
:1018F00093F102C194F103C195F11A0E64EC0BF05F
:10190000E8CF00F11B0E64EC0BF0E8CF01F11C0EE8
:1019100064EC0BF0E8CF02F11D0E64EC0BF0E8CFA5
:1019200003F1010103AFC3EF0CF015EC31F01A0E17
:101930000C6E00C10BF04DEC0BF01B0E0C6E01C1D8
:101940000BF04DEC0BF01C0E0C6E02C10BF04DECCD
:101950000BF01D0E0C6E03C10BF04DEC0BF01A0ECC
:1019600064EC0BF0E8CF00F11B0E64EC0BF0E8CF59
:1019700001F11C0E64EC0BF0E8CF02F11D0E64ECDB
:101980000BF0E8CF03F100C196F101C197F102C15C
:1019900098F103C199F1240EAC6E900EAB6E240E3B
:1019A000AC6E080EB86E000EB06E1F0EAF6E040166
:1019B000806B816B0F01900EAB6E0F019D8A03014E
:1019C000806B816BC26B8B9252EC36F052EC36F02E
:1019D00034EC38F030EC34F0200E64EC0BF0E8CF4F
:1019E0002FF505012F51FF0AD8A4FEEF0CF02F6B45
:1019F000200E0C6E2FC50BF04DEC0BF00501010E07
:101A0000306F3C0E316F250E64EC0BF0E8CF00F127
:101A1000260E64EC0BF0E8CF01F1270E64EC0BF01E
:101A2000E8CF02F1280E64EC0BF0E8CF03F10101DE
:101A300003AF35EF0DF015EC31F0250E0C6E00C143
:101A40000BF04DEC0BF0260E0C6E01C10BF04DECC3
:101A50000BF0270E0C6E02C10BF04DEC0BF0280EB4
:101A60000C6E03C10BF04DEC0BF000C157F501C13A
:101A700058F502C159F503C15AF500C15BF501C122
:101A80005CF502C15DF503C15EF5290E64EC0BF057
:101A9000E8CF5FF5050160515F5DD8A05FC560F5D7
:101AA000210E64EC0BF0E8CF00F1220E64EC0BF099
:101AB000E8CF01F1230E64EC0BF0E8CF02F1240E25
:101AC00064EC0BF0E8CF03F1010103AF96EF0DF0EA
:101AD00015EC31F0210E0C6E00C10BF04DEC0BF04B
:101AE000220E0C6E01C10BF04DEC0BF0230E0C6EB0
:101AF00002C10BF04DEC0BF0240E0C6E03C10BF089
:101B00004DEC0BF0210E64EC0BF0E8CF00F1220E4F
:101B100064EC0BF0E8CF01F1230E64EC0BF0E8CF9E
:101B200002F1240E64EC0BF0E8CF03F100C161F583
:101B300001C162F502C163F503C164F578EC33F0CD
:101B40005EEC32F0B6EC31F01590C70E64EC0BF0A1
:101B5000E8CF00F1010100B1B1EF0DF01592B2EF45
:101B60000DF0158281AAC0EF0DF015B4BBEF0DF09A
:101B70001580C0EF0DF073EC38F015A0DAEF38F0F7
:101B800007900001F28EF28C12AE03D012BC6EEF01
:101B900019F007B027EF2DF00FB023EF26F010BE9D
:101BA00023EF26F012B823EF26F000011650010AA9
:101BB000D8B41CEF1EF081BAE6EF0DF0000116500C
:101BC000040AD8B41AEF1CF0ECEF0DF00001165027
:101BD000040AD8B458EF1EF00301805181197F0B1D
:101BE000D8B427EF2DF013EE00F081517F0BE126E2
:101BF000812BE7CFE8FFE00BD8B427EF2DF023EEE1
:101C000082F0C2513F0BD926E7CFDFFFC22BDF5056
:101C1000780AD8A427EF2DF0078092C100F193C174
:101C200001F194C102F195C103F10101040E046FA9
:101C3000000E056F000E066F000E076F00EC30F00F
:101C400000AF2CEF0EF00101030E926F000E936FA8
:101C5000000E946F000E956F03018251720AD8B482
:101C6000A4EF25F08251520AD8B4A4EF25F0825196
:101C7000750AD8B4A4EF25F08251680AD8B4AAEF47
:101C80000EF08251630AD8B4E1EF29F08251690A5B
:101C9000D8B462EF21F082517A0AD8B475EF22F0FD
:101CA0008251490AD8B401EF21F08251500AD8B4C8
:101CB0001FEF20F08251700AD8B462EF20F08251F9
:101CC000540AD8B48DEF20F08251740AD8B4D3EFFF
:101CD00020F08251410AD8B4AFEF0FF082514B0A85
:101CE000D8B4ACEF0EF082516D0AD8B41FEF14F0E7
:101CF00082514D0AD8B438EF14F08251730AD8B427
:101D0000D4EF24F08251530AD8B439EF25F0825130
:101D10004C0AD8B4C7EF14F08251590AD8B470EF06
:101D200013F012AE01D0128C18EF2AF0040114EE59
:101D300000F080517F0BE12682C4E7FF802B120068
:101D400004010D0E826F96EC0EF00A0E826F96EC77
:101D50000EF0120016EF2AF004014B0E826F96EC83
:101D60000EF004012C0E826F96EC0EF081B802D0BA
:101D700036B630D003018351430AD8B4F1EF0EF0E8
:101D800003018351630AD8B4F3EF0EF003018351CA
:101D9000520AD8B4F5EF0EF003018351720AD8B499
:101DA000F7EF0EF003018351470AD8B4F9EF0EF0B4
:101DB00003018351670AD8B4FBEF0EF0030183518E
:101DC000540AD8B4FDEF0EF003018351740AD8B45D
:101DD0006DEF0FF003018351550AD8B4FFEF0EF0F9
:101DE00083D036807BD0369079D0368277D03692C9
:101DF00075D0368473D0369471D036866FD084C354
:101E000030F185C331F186C332F187C333F101016B
:101E1000296B63EC31F0DAEC30F000C104F101C160
:101E200005F102C106F103C107F156EC31F0200EB5
:101E3000F86EF76AF66A0900F5CF2CF10900F5CFC4
:101E40002DF10900F5CF2EF10900F5CF2FF1090092
:101E5000F5CF30F10900F5CF31F10900F5CF32F1BE
:101E60000900F5CF33F10101296B63EC31F0DAECB5
:101E700030F000EC30F00101006746EF0FF0016731
:101E800046EF0FF0026746EF0FF0036701D025D051
:101E900004014E0E826F96EC0EF004016F0E826FFD
:101EA00096EC0EF004014D0E826F96EC0EF00401DC
:101EB000610E826F96EC0EF00401740E826F96EC48
:101EC0000EF00401630E826F96EC0EF00401680EB2
:101ED000826F96EC0EF016EF2AF03696CD0E0C6E51
:101EE00036C00BF04DEC0BF0CD0E64EC0BF0E8CFF0
:101EF00036F036B006D00401630E826F96EC0EF019
:101F000005D00401430E826F96EC0EF036B206D077
:101F10000401720E826F96EC0EF005D00401520E91
:101F2000826F96EC0EF036B406D00401670E826F15
:101F300096EC0EF005D00401470E826F96EC0EF081
:101F400036B606D00401740E826F96EC0EF005D002
:101F50000401540E826F96EC0EF016EF2AF0040185
:101F6000410E826F96EC0EF003018351310AD8B412
:101F700090EF12F003018351320AD8B4C0EF11F090
:101F800003018351330AD8B449EF11F0030183519F
:101F9000340AD8B439EF10F003018351350AD8B4AC
:101FA000D9EF0FF004013F0E826F96EC0EF016EFA2
:101FB0002AF003018451300AD8B4FFEF0FF0030177
:101FC0008451310AD8B402EF10F003018451650A3C
:101FD000D8B4F3EF0FF003018451640AD8B4F6EFDC
:101FE0000FF003EF10F03790F7EF0FF03780FB0E94
:101FF0000C6E37C00BF04DEC0BF003EF10F08B9034
:1020000003EF10F08B800401350E826F96EC0EF01A
:1020100004012C0E826F96EC0EF08BB017EF10F0CF
:102020000401300E826F96EC0EF01CEF10F00401EC
:10203000310E826F96EC0EF004012C0E826F96EC3E
:102040000EF0FB0E64EC0BF0E8CF37F037A030EF6A
:1020500010F00401640E826F96EC0EF035EF10F074
:102060000401650E826F96EC0EF037EF10F016EF5C
:102070002AF0CC0E64EC0BF0E8CF0BF004012C0E30
:10208000826F96EC0EF003018451310AD8B45DEFF3
:1020900010F003018451300AD8B45FEF10F003014F
:1020A00084514D0AD8B469EF10F003018451540AE9
:1020B000D8B470EF10F087EF10F08A8401D08A94C2
:1020C0000BAE04D00BAC02D00BBA21D0E00E0B1239
:1020D00018D01F0E0B168539E844E00B0B1211D0F7
:1020E000E00E0B1656EC31F085C332F186C333F1A6
:1020F0000101296B63EC31F0DAEC30F000511F0B79
:102100000B12CC0E0C6E0BC00BF04DEC0BF004015F
:10211000340E826F96EC0EF004012C0E826F96EC5A
:102120000EF0CC0E64EC0BF0E8CF1DF08AB406D0B4
:102130000401300E826F96EC0EF005D00401310ED2
:10214000826F96EC0EF004012C0E826F96EC0EF06E
:102150001D38E840070BE8CF82F40401300E8227D7
:1021600096EC0EF004012C0E826F96EC0EF015EC3E
:1021700031F01D501F0BE8CF00F19EEC30F032C162
:1021800082F40401300E822796EC0EF033C182F403
:102190000401300E822796EC0EF004012C0E826FA3
:1021A00096EC0EF015EC31F030C000F100AF0BD022
:1021B000FF0E016FFF0E026FFF0E036F04012D0E65
:1021C000826F96EC0EF09EEC30F031C182F4040187
:1021D000300E822796EC0EF032C182F40401300EEC
:1021E000822796EC0EF033C182F40401300E822770
:1021F00096EC0EF004012C0E826F96EC0EF015ECAE
:1022000031F02FC000F19EEC30F031C182F40401B6
:10221000300E822796EC0EF032C182F40401300EAB
:10222000822796EC0EF033C182F40401300E82272F
:1022300096EC0EF004012C0E826F96EC0EF015EC6D
:1022400031F031C000F100AF0BD0FF0E016FFF0E77
:10225000026FFF0E036F04012D0E826F96EC0EF0DD
:102260009EEC30F031C182F40401300E822796ECEE
:102270000EF032C182F40401300E822796EC0EF08B
:1022800033C182F40401300E822796EC0EF016EF73
:102290002AF0CB0E64EC0BF0E8CF0BF004012C0E0F
:1022A000826F96EC0EF003018451450AD8B46DEFAD
:1022B00011F003018451440AD8B470EF11F0030106
:1022C0008451300AD8B473EF11F003018451310AFC
:1022D000D8B477EF11F082EF11F00B9E7CEF11F084
:1022E0000B8E7CEF11F0FC0E0B167CEF11F0FC0E48
:1022F0000B160B807CEF11F0CB0E0C6E0BC00BF0AD
:102300004DEC0BF00401330E826F96EC0EF00401DD
:102310002C0E826F96EC0EF0CB0E64EC0BF0E8CF37
:102320001CF01CBE9BEF11F00401450E826F96EC71
:102330000EF0A0EF11F00401440E826F96EC0EF047
:1023400004012C0E826F96EC0EF00401300E826FA9
:1023500096EC0EF004012C0E826F96EC0EF01CB081
:10236000B9EF11F00401300E826F96EC0EF0BEEF63
:1023700011F00401310E826F96EC0EF016EF2AF088
:10238000CA0E64EC0BF0E8CF0BF004012C0E826F48
:1023900096EC0EF003018451450AD8B4FCEF11F01D
:1023A00003018451440AD8B4FFEF11F003018451B2
:1023B0004D0AD8B408EF12F003018451410AD8B491
:1023C00002EF12F003018451460AD8B405EF12F06F
:1023D00003018451560AD8B410EF12F0030184515E
:1023E000500AD8B41BEF12F003018451520AD8B43A
:1023F0001EEF12F027EF12F00B9E21EF12F00B8E62
:1024000021EF12F00B9C21EF12F00B8C21EF12F058
:10241000FC0E0B1685C3E8FF030B0B1221EF12F025
:10242000C70E0B1685C3E8FF070BE846E846E846EB
:102430000B1221EF12F00B8421EF12F00B9421EF1D
:1024400012F0CA0E0C6E0BC00BF04DEC0BF0CA0E66
:1024500064EC0BF0E8CF1BF00401320E826F96ECB7
:102460000EF004012C0E826F96EC0EF01BBE40EFB6
:1024700012F00401450E826F96EC0EF045EF12F05B
:102480000401440E826F96EC0EF004012C0E826F54
:1024900096EC0EF01BC0E8FF030BE8CF82F40401BA
:1024A000300E822796EC0EF004012C0E826F96EC13
:1024B0000EF01BBC63EF12F00401410E826F96EC2C
:1024C0000EF068EF12F00401460E826F96EC0EF0EB
:1024D00004012C0E826F96EC0EF01BC0E8FF380B47
:1024E000E842E842E842E8CF82F40401300E822755
:1024F00096EC0EF004012C0E826F96EC0EF01BB4DD
:1025000089EF12F00401520E826F96EC0EF08EEFFE
:1025100012F00401500E826F96EC0EF016EF2AF0C6
:10252000C90E64EC0BF0E8CF0BF004012C0E826FA7
:1025300096EC0EF003018451450AD8B4AEEF12F0C8
:1025400003018451440AD8B4B1EF12F0030184515D
:102550004D0AD8B4B4EF12F0C2EF12F00B9EBCEFEC
:1025600012F00B8EBCEF12F0F80E0B1685C3E8FFCD
:10257000070B0B12BCEF12F0C90E0C6E0BC00BF068
:102580004DEC0BF00401310E826F96EC0EF004015D
:102590002C0E826F96EC0EF0C90E64EC0BF0E8CFB7
:1025A0001AF01ABE06D00401450E826F96EC0EF0AA
:1025B00005D00401440E826F96EC0EF004012C0E3F
:1025C000826F96EC0EF01AC0E8FF070BE8CF82F49A
:1025D0000401300E822796EC0EF004012C0E826F5F
:1025E00096EC0EF0078015EC31F02BC0E8FF003BB5
:1025F00000430043030B9EEC30F033C182F404012E
:10260000300E822796EC0EF004012C0E826F96ECB1
:102610000EF015EC31F02BC001F1019F019D2CC093
:1026200000F101019EEC30F02FC182F40401300E64
:10263000822796EC0EF030C182F40401300E82271E
:1026400096EC0EF031C182F40401300E822796EC34
:102650000EF032C182F40401300E822796EC0EF0A7
:1026600033C182F40401300E822796EC0EF004018F
:102670002C0E826F96EC0EF015EC31F02DC001F1AE
:102680002EC000F1D89001330033D89001330033CD
:1026900001019EEC30F02FC182F40401300E82273C
:1026A00096EC0EF030C182F40401300E822796ECD5
:1026B0000EF031C182F40401300E822796EC0EF048
:1026C00032C182F40401300E822796EC0EF033C141
:1026D00082F40401300E822796EC0EF016EF2AF0F9
:1026E000FC0E64EC0BF0E8CF0BF003018351520AAF
:1026F000D8B4A7EF13F003018351720AD8B4AAEF3C
:1027000013F003018351500AD8B4ADEF13F0030165
:102710008351700AD8B4B0EF13F003018351550A06
:10272000D8B4B3EF13F003018351750AD8B4B6EFF0
:1027300013F003018351430AD8B4BFEF13F0030130
:102740008351630AD8B4C2EF13F0CBEF13F00B90B0
:10275000C5EF13F00B80C5EF13F00B92C5EF13F02C
:102760000B82C5EF13F00B94C5EF13F00B84C5EF8C
:1027700013F00B96C5EF13F00B86C5EF13F00B9813
:10278000C5EF13F00B88C5EF13F0FC0E0C6E0BC0F9
:102790000BF04DEC0BF00401590E826F96EC0EF02D
:1027A0001190119211941198FC0E64EC0BF0E8CF8B
:1027B0000BF00BA011800BA211820BA411840BA8AB
:1027C000118811A0EBEF13F00401520E826F96EC0A
:1027D0000EF0F0EF13F00401720E826F96EC0EF023
:1027E00011A8FAEF13F00401430E826F96EC0EF07D
:1027F000FFEF13F00401630E826F96EC0EF011A24E
:1028000009EF14F00401500E826F96EC0EF00EEFFB
:1028100014F00401700E826F96EC0EF011A418EF04
:1028200014F00401550E826F96EC0EF01DEF14F0BB
:102830000401750E826F96EC0EF016EF2AF004017B
:102840006D0E826F96EC0EF003018351300AD8B4FE
:1028500077EF14F003018351310AD8B48AEF14F0F2
:1028600003018351320AD8B49DEF14F018EF2AF017
:1028700004014D0E826F96EC0EF056EC31F084C3DD
:1028800031F185C332F186C333F10101296B63EC69
:1028900031F0DAEC30F003018351300AD8B45FEF45
:1028A00014F003018351310AD8B467EF14F0030127
:1028B0008351320AD8B46FEF14F018EF2AF0FD0EEE
:1028C0000C6E00C10BF04DEC0BF077EF14F0FE0E28
:1028D0000C6E00C10BF04DEC0BF08AEF14F0FF0E04
:1028E0000C6E00C10BF04DEC0BF09DEF14F00401E9
:1028F000300E826F96EC0EF004012C0E826F96EC77
:102900000EF015EC31F0FD0E64EC0BF0E8CF00F1A9
:10291000AEEF14F00401310E826F96EC0EF004015C
:102920002C0E826F96EC0EF015EC31F0FE0E64EC7E
:102930000BF0E8CF00F1AEEF14F00401320E826F1D
:1029400096EC0EF015EC31F004012C0E826F96EC33
:102950000EF0FF0E64EC0BF0E8CF00F19EEC30F0CF
:1029600031C182F40401300E822796EC0EF032C1A0
:1029700082F40401300E822796EC0EF033C182F40B
:102980000401300E822796EC0EF016EF2AF00301B8
:102990008351300AD8B41BEF1AF003018351310A76
:1029A000D8B448EF1BF003018351320AD8B4B6EF14
:1029B0001BF003018351330AD8B4C6EF1BF00301A7
:1029C0008351340AD8B421EF1CF003018351350A36
:1029D000D8B470EF1EF003018351360AD8B49EEFCD
:1029E0001EF003018351370AD8B4F3EF17F0030147
:1029F0008351380AD8B491EF18F003018351440A87
:102A0000D8B41FEF16F003018351640AD8B43FEF26
:102A100016F003018351460AD8B475EF1DF0030187
:102A200083514D0AD8B46CEF16F0030183516D0A3F
:102A3000D8B486EF16F0030183515A0AD8B4C2EF16
:102A40001AF003018351490AD8B49EEF1FF0030125
:102A50008351500AD8B4D0EF1EF003018351540AB9
:102A6000D8B449EF1FF003018351630AD8B4A6EF2D
:102A700016F003018351430AD8B49EEF17F0030107
:102A80008351730AD8B4A4EF16F003018351610A8D
:102A9000D8B46CEF15F003018351650AD8B46BEF1D
:102AA0001AF003018351450AD8B479EF1AF00301F3
:102AB0008351620AD8B487EF1AF003018351420AA6
:102AC000D8B495EF1AF003018351760AD8B4A3EF76
:102AD0001AF0D8A418EF2AF004014C0E826F96EC7D
:102AE0000EF00401610E826F96EC0EF05EEC32F097
:102AF00004012C0E826F96EC0EF015EC31F0AFC590
:102B000000F101019EEC30F031C182F40401300E7D
:102B1000822796EC0EF032C182F40401300E822737
:102B200096EC0EF033C182F40401300E822796EC4D
:102B30000EF004012C0E826F96EC0EF015EC31F0C5
:102B4000B0C500F101019EEC30F031C182F4040106
:102B5000300E822796EC0EF032C182F40401300E62
:102B6000822796EC0EF033C182F40401300E8227E6
:102B700096EC0EF004012C0E826F96EC0EF015EC24
:102B800031F0B1C500F101019EEC30F031C182F4A9
:102B90000401300E822796EC0EF032C182F404015B
:102BA000300E822796EC0EF033C182F40401300E11
:102BB000822796EC0EF004012C0E826F96EC0EF03C
:102BC00015EC31F0B2C500F101019EEC30F031C1DD
:102BD00082F40401300E822796EC0EF032C182F4AA
:102BE0000401300E822796EC0EF033C182F404010A
:102BF000300E822796EC0EF004012C0E826F96ECBC
:102C00000EF015EC31F0B6C500F101019EEC30F08C
:102C100031C182F40401300E822796EC0EF032C1ED
:102C200082F40401300E822796EC0EF033C182F458
:102C30000401300E822796EC0EF0CCEF1EF003015B
:102C40008451300AD8B42BEF16F003018451310AB5
:102C5000D8B42FEF16F01592159630EF16F01582B6
:102C6000C70E64EC0BF0E8CF00F10101008115A262
:102C70000091C70E0C6E00C10BF04DEC0BF0C70EAF
:102C800064EC0BF0E8CF00F1010100B14BEF16F05E
:102C900015924CEF16F0158204014C0E826F96ECE3
:102CA0000EF00401640E826F96EC0EF004012C0EFF
:102CB000826F96EC0EF015B265EF16F00401300E3F
:102CC000826F96EC0EF06AEF16F00401310E826FFF
:102CD00096EC0EF016EF2AF056EC31F084C333F187
:102CE00063EC31F0DAEC30F0200E0C6E00C10BF02A
:102CF0004DEC0BF000C12FF505012F51000A06E045
:102D000005012F51010A02E0F8EC32F004014C0EEB
:102D1000826F96EC0EF004014D0E826F96EC0EF071
:102D200004012C0E826F96EC0EF015EC31F02FC5DD
:102D300000F19EEC30F033C182F40401300E8227A2
:102D400096EC0EF0CCEF1EF0DAEF38F004014C0EEA
:102D5000826F96EC0EF00401630E826F96EC0EF01B
:102D6000B6EC31F004012C0E826F96EC0EF0BBEC49
:102D700016F0CCEF1EF015EC31F0B5C500F10101F5
:102D8000003B0F0E00179EEC30F033C182F40401BB
:102D9000300E822796EC0EF0B5C500F101010F0E42
:102DA000010100179EEC30F033C182F40401300EB3
:102DB000822796EC0EF004012D0E826F96EC0EF039
:102DC000B4C500F10101003B0F0E00179EEC30F07E
:102DD00033C182F40401300E822796EC0EF0B4C5A4
:102DE00000F101010F0E010100179EEC30F033C11C
:102DF00082F40401300E822796EC0EF004012D0EB1
:102E0000826F96EC0EF0B3C500F10101003B0F0E8E
:102E100000179EEC30F033C182F40401300E82279B
:102E200096EC0EF0B3C500F101010F0E0101001781
:102E30009EEC30F033C182F40401300E822796EC10
:102E40000EF00401200E826F96EC0EF0B2C500F178
:102E50000F0E010100179EEC30F033C182F4040123
:102E6000300E822796EC0EF00401200E826F96EC55
:102E70000EF0B1C500F101010101003B0F0E00177A
:102E80009EEC30F033C182F40401300E822796ECC0
:102E90000EF0B1C500F101010F0E010100179EEC0B
:102EA00030F033C182F40401300E822796EC0EF02C
:102EB00004013A0E826F96EC0EF0B0C500F10101EC
:102EC000003B0F0E00179EEC30F033C182F404017A
:102ED000300E822796EC0EF0B0C500F101010F0E06
:102EE000010100179EEC30F033C182F40401300E72
:102EF000822796EC0EF004013A0E826F96EC0EF0EB
:102F0000AFC500F10101003B0F0E00179EEC30F041
:102F100033C182F40401300E822796EC0EF0AFC567
:102F200000F101010F0E00179EEC30F033C182F466
:102F30000401300E822796EC0EF0120084C3E8FFE5
:102F40000F0BE83AE8CFB5F585C3E8FF0F0B050195
:102F5000B51387C3E8FF0F0BE83AE8CFB4F588C391
:102F6000E8FF0F0B0501B4138AC3E8FF0F0BE83A23
:102F7000E8CFB3F58BC3E8FF0F0B0501B3138DC387
:102F8000E8FF0F0BE8CFB2F58FC3E8FF0F0BE83A6D
:102F9000E8CFB1F590C3E8FF0F0B0501B11392C361
:102FA000E8FF0F0BE83AE8CFB0F593C3E8FF0F0B4B
:102FB0000501B01395C3E8FF0F0BE83AE8CFAFF572
:102FC00096C3E8FF0F0B0501AF1311EC32F00401BB
:102FD0004C0E826F96EC0EF00401430E826F96EC5D
:102FE0000EF0B0EF16F0078404014C0E826F96ECE1
:102FF0000EF00401370E826F96EC0EF004012C0ED9
:10300000826F96EC0EF005012E51130A06E00501C1
:103010002E51170A0DE08EEF18F00101000E006F1F
:10302000000E016F100E026F000E036F21EF18F0FB
:103030000101000E006F000E016F000E026F010E05
:10304000036F9EEC30F02AC182F40401300E822717
:1030500096EC0EF02BC182F40401300E822796EC20
:103060000EF02CC182F40401300E822796EC0EF093
:103070002DC182F40401300E822796EC0EF02EC191
:1030800082F40401300E822796EC0EF02FC182F4F8
:103090000401300E822796EC0EF030C182F4040158
:1030A000300E822796EC0EF031C182F40401300E0E
:1030B000822796EC0EF032C182F40401300E822792
:1030C00096EC0EF033C182F40401300E822796ECA8
:1030D0000EF004012C0E826F96EC0EF00101200E12
:1030E000006F000E016F000E026F000E036F9EEC6A
:1030F00030F031C182F40401300E822796EC0EF0DC
:1031000032C182F40401300E822796EC0EF033C1F6
:1031100082F40401300E822796EC0EF00794CCEF77
:103120001EF00501216B226B236B246B04014C0EF6
:10313000826F96EC0EF00401380E826F96EC0EF062
:1031400004012C0E826F96EC0EF00101200E006F30
:10315000000E016F000E026F000E036F9EEC30F048
:103160002AC182F40401300E822796EC0EF02BC1A6
:1031700082F40401300E822796EC0EF02CC182F40A
:103180000401300E822796EC0EF02DC182F404016A
:10319000300E822796EC0EF02EC182F40401300E20
:1031A000822796EC0EF02FC182F40401300E8227A4
:1031B00096EC0EF030C182F40401300E822796ECBA
:1031C0000EF031C182F40401300E822796EC0EF02D
:1031D00032C182F40401300E822796EC0EF033C126
:1031E00082F40401300E822796EC0EF004012C0EBE
:1031F000826F96EC0EF025C500F126C501F127C5BA
:1032000002F128C503F10101200E046F000E056FC5
:10321000000E066F000E076F31EC30F000C133F581
:1032200001C134F502C135F503C136F59EEC30F02D
:103230002AC182F40401300E822796EC0EF02BC1D5
:1032400082F40401300E822796EC0EF02CC182F439
:103250000401300E822796EC0EF02DC182F4040199
:10326000300E822796EC0EF02EC182F40401300E4F
:10327000822796EC0EF02FC182F40401300E8227D3
:1032800096EC0EF030C182F40401300E822796ECE9
:103290000EF031C182F40401300E822796EC0EF05C
:1032A00032C182F40401300E822796EC0EF033C155
:1032B00082F40401300E822796EC0EF0A0EC0EF0A2
:1032C000050133676BEF19F034676BEF19F0356761
:1032D0006BEF19F0366702D00AEF1AF0129E129CBB
:1032E00021C500F122C501F123C502F124C503F176
:1032F000899A400EC76E200EC66E9E96C69E0B0E15
:10330000C96EFF0E9EB602D0E82EFCD79E96C69ED2
:1033100002C1C9FFFF0E9EB602D0E82EFCD79E96D2
:10332000C69E01C1C9FFFF0E9EB602D0E82EFCD793
:103330009E96C69E00C1C9FFFF0E9EB602D0E82E23
:10334000FCD79E96C69EC952FF0E9EB602D0E82EAE
:10335000FCD70501200E326F040114EE00F08051FD
:103360007F0BE1269E96C69EC952FF0E9EB602D0E6
:10337000E82EFCD7C9CFE7FF0401802B0501322FCF
:10338000ACEF19F0898A33C500F134C501F135C5B8
:1033900002F136C503F10101010E046F000E056F45
:1033A000000E066F000E076F00EC30F000C133F521
:1033B00001C134F502C135F503C136F505013367A6
:1033C000E9EF19F03467E9EF19F03567E9EF19F023
:1033D000366702D00AEF1AF021C500F122C501F1CB
:1033E00023C502F124C503F10101200E046F000E74
:1033F000056F000E066F000E076F05EC30F000C180
:1034000021F501C122F502C123F503C124F5128E75
:1034100018EF2AF00401450E826F96EC0EF00401BD
:103420004F0E826F96EC0EF00401460E826F96EC02
:103430000EF0CCEF1EF0078434EC38F015EC31F0D0
:103440002DC500F19EEC30F004014C0E826F96EC1D
:103450000EF00401300E826F96EC0EF004012C0E7B
:10346000826F96EC0EF031C182F40401300E822797
:1034700096EC0EF032C182F40401300E822796ECF5
:103480000EF033C182F40401300E822796EC0EF068
:1034900004012C0E826F96EC0EF015EC31F02EC567
:1034A00000F19EEC30F031C182F40401300E82272D
:1034B00096EC0EF032C182F40401300E822796ECB5
:1034C0000EF033C182F40401300E822796EC0EF028
:1034D0000794CCEF1EF004014C0E826F96EC0EF0B8
:1034E0000401650E826F96EC0EF0D4EC33F0CCEF55
:1034F0001EF004014C0E826F96EC0EF00401450E96
:10350000826F96EC0EF0EBEC33F0CCEF1EF0040182
:103510004C0E826F96EC0EF00401620E826F96ECF8
:103520000EF019EC34F0CCEF1EF004014C0E826F5B
:1035300096EC0EF00401420E826F96EC0EF002EC57
:1035400034F0CCEF1EF004014C0E826F96EC0EF0BE
:103550000401760E826F96EC0EF004012C0E826F41
:1035600096EC0EF010A807D00401310E826F96EC95
:103570000EF0CCEF1EF00401300E826F96EC0EF0D0
:10358000CCEF1EF004014C0E826F96EC0EF004019D
:103590005A0E826F96EC0EF004012C0E826F96ECA0
:1035A0000EF034EC38F015EC31F005012E51130A11
:1035B00006E005012E51170A0DE0F3EF1AF00101A4
:1035C000000E006F000E016F100E026F000E036FF1
:1035D000F3EF1AF00101000E006F000E016F000EF4
:1035E000026F010E036F0101200E046F000E056FC4
:1035F000000E066F000E076F31EC30F09EEC30F0DD
:103600002AC182F40401300E822796EC0EF02BC101
:1036100082F40401300E822796EC0EF02CC182F465
:103620000401300E822796EC0EF02DC182F40401C5
:10363000300E822796EC0EF02EC182F40401300E7B
:10364000822796EC0EF02FC182F40401300E8227FF
:1036500096EC0EF030C182F40401300E822796EC15
:103660000EF031C182F40401300E822796EC0EF088
:1036700032C182F40401300E822796EC0EF033C181
:1036800082F40401300E822796EC0EF0CCEF1EF08F
:10369000078404014C0E826F96EC0EF00401310E8B
:1036A000826F96EC0EF004012C0E826F96EC0EF0F9
:1036B00025C500F126C501F127C502F128C503F192
:1036C0000101200E046F000E056F000E066F000E44
:1036D000076F31EC30F09EEC30F02AC182F4040127
:1036E000300E822796EC0EF02BC182F40401300ECE
:1036F000822796EC0EF02CC182F40401300E822752
:1037000096EC0EF02DC182F40401300E822796EC67
:103710000EF02EC182F40401300E822796EC0EF0DA
:103720002FC182F40401300E822796EC0EF030C1D6
:1037300082F40401300E822796EC0EF031C182F43F
:103740000401300E822796EC0EF032C182F404019F
:10375000300E822796EC0EF033C182F40401300E55
:10376000822796EC0EF00794CCEF1EF0078404013C
:103770004C0E826F96EC0EF00401320E826F96ECC6
:103780000EF008EC36F00794CCEF1EF0078437B04B
:10379000CCEF1BF0DFEF1BF0010E166E04014C0E98
:1037A000826F96EC0EF00401330E826F96EC0EF0F1
:1037B00065EC36F0000E166E079453EF1BF0020E08
:1037C000166E65EC36F08B800501010E306F3C0EF5
:1037D000316F01015E6B5F6B606B616B626B636B82
:1037E000646B656B666B676B686B696B536B546B73
:1037F000CF6ACE6A0F9A0F9C0F9E030E166E0401BD
:103800004C0E826F96EC0EF00401330E826F96EC34
:103810000EF004012C0E826F96EC0EF004012D0EBA
:10382000826F96EC0EF00401310E826F96EC0EF072
:1038300016EF2AF065EC36F0000E166E8B9018EF3E
:103840002AF0078404014C0E826F96EC0EF00401FE
:10385000340E826F96EC0EF004012C0E826F96EC03
:103860000EF056EC31F084C32AF185C32BF186C3E8
:103870002CF187C32DF188C32EF189C32FF18AC3A0
:1038800030F18BC331F18CC332F18DC333F10101BF
:10389000296B63EC31F0DAEC30F0200E046F000E8F
:1038A000056F000E066F000E076F11EC30F000C1BF
:1038B00021F501C122F502C123F503C124F5E7EC8E
:1038C00037F038C5AFF539C5B0F53AC5B1F53BC5E8
:1038D000B2F53CC5B3F53DC5B4F53EC5B5F5BBEC99
:1038E00016F004012C0E826F96EC0EF03FC500F12D
:1038F00040C501F141C502F142C503F10101000ECD
:10390000046F000E056F010E066F000E076F31EC9D
:1039100030F09EEC30F0296790EF1CF095EF1CF032
:1039200004012D0E826F96EC0EF030C182F404017A
:10393000300E822796EC0EF031C182F40401300E75
:10394000822796EC0EF004012E0E826F96EC0EF09C
:1039500032C182F40401300E822796EC0EF033C19E
:1039600082F40401300E822796EC0EF004012C0E36
:10397000826F96EC0EF015EC31F043C500F144C5B2
:1039800001F142EC2BF004012C0E826F96EC0EF04C
:1039900015EC31F045C500F19EEC30F031C182F4F8
:1039A0000401300E822796EC0EF032C182F404013D
:1039B000300E822796EC0EF033C182F40401300EF3
:1039C000822796EC0EF004012C0E826F96EC0EF01E
:1039D00037C5E8FFE8B806D00401300E826F96ECD8
:1039E0000EF005D00401310E826F96EC0EF004014A
:1039F0002C0E826F96EC0EF037C5E8FFE8BA06D0C1
:103A00000401300E826F96EC0EF06CD00401310E82
:103A1000826F96EC0EF004012C0E826F96EC0EF085
:103A200047C500F148C501F149C502F14AC503F196
:103A3000C0EC30F061EC2EF004012C0E826F96EC9D
:103A40000EF04BC500F14CC501F14DC502F14EC55C
:103A500003F10101000E046F000E056F010E066FE9
:103A6000000E076F31EC30F09EEC30F029673BEF31
:103A70001DF040EF1DF004012D0E826F96EC0EF04C
:103A800030C182F40401300E822796EC0EF031C171
:103A900082F40401300E822796EC0EF004012E0E03
:103AA000826F96EC0EF032C182F40401300E822750
:103AB00096EC0EF033C182F40401300E822796ECAE
:103AC0000EF004012C0E826F96EC0EF04FC500F143
:103AD00050C501F151C502F152C503F1C0EC30F0FF
:103AE00061EC2EF00794CCEF1EF056EC31F085C35C
:103AF0002AF186C32BF187C32CF188C32DF189C32A
:103B00002EF18AC32FF18BC330F18CC331F18DC3F9
:103B100032F18EC333F10101296B63EC31F0DAEC41
:103B200030F00101010E046F000E056F000E066FEC
:103B3000000E076F00EC30F0100E046F000E056FE2
:103B4000000E066F000E076F11EC30F000C129F572
:103B500001C12AF502C12BF503C12CF58FEC35F01C
:103B600004014C0E826F96EC0EF00401460E826F3B
:103B700096EC0EF004012C0E826F96EC0EF025C52B
:103B800000F126C501F127C502F128C503F10101A5
:103B9000100E046F000E056F000E066F000E076F0B
:103BA00031EC30F09EEC30F02AC182F40401300E8A
:103BB000822796EC0EF02BC182F40401300E82278E
:103BC00096EC0EF02CC182F40401300E822796ECA4
:103BD0000EF02DC182F40401300E822796EC0EF017
:103BE0002EC182F40401300E822796EC0EF02FC114
:103BF00082F40401300E822796EC0EF030C182F47C
:103C00000401300E822796EC0EF031C182F40401DB
:103C1000300E822796EC0EF032C182F40401300E91
:103C2000822796EC0EF033C182F40401300E822715
:103C300096EC0EF0CCEF1EF037B021EF1EF0020E26
:103C4000166E65EC36F000011650020AD8B43FEF4C
:103C50001EF005012F51010AD8B435EF1EF015B240
:103C60003AEF1EF081BA3AEF1EF0000E166E158480
:103C700018EF2AF0050E166E1584DAEF38F08B80F7
:103C800001015E6B5F6B606B616B626B636B646B9E
:103C9000656B666B676B686B696B536B546BCF6A54
:103CA000CE6A0F9A0F9C0F9E030E166E18EF2AF025
:103CB00065EC36F005012F51010AD8B466EF1EF00D
:103CC00015B26BEF1EF081BA6BEF1EF0000E166E90
:103CD000158418EF2AF0050E166E1584DAEF38F009
:103CE00004014C0E826F96EC0EF00401350E826FCB
:103CF00096EC0EF004012C0E826F96EC0EF015EC93
:103D000031F00784B9C500F107949EEC30F031C161
:103D100082F40401300E822796EC0EF032C182F458
:103D20000401300E822796EC0EF033C182F40401B8
:103D3000300E822796EC0EF0CCEF1EF028EC36F019
:103D400015EC31F037C500F19EEC30F004014C0E5B
:103D5000826F96EC0EF00401360E826F96EC0EF038
:103D600004012C0E826F96EC0EF031C182F4040136
:103D7000300E822796EC0EF032C182F40401300E30
:103D8000822796EC0EF033C182F40401300E8227B4
:103D900096EC0EF0CCEF1EF0A0EC0EF018EF2AF02F
:103DA00004014C0E826F96EC0EF00401500E826FEF
:103DB00096EC0EF004012C0E826F96EC0EF085C38B
:103DC0002AF186C32BF187C32CF188C32DF189C357
:103DD0002EF18AC32FF18BC330F18CC331F18DC327
:103DE00032F18EC333F1010163EC31F0DAEC30F0E3
:103DF00003018451530A0DE0030184514D0A38E058
:103E00000401780E826F96EC0EF0A0EC0EF018EF25
:103E10002AF00401530E826F96EC0EF0250E0C6E04
:103E200000C10BF04DEC0BF0260E0C6E01C10BF037
:103E30004DEC0BF0270E0C6E02C10BF04DEC0BF0AD
:103E4000280E0C6E03C10BF04DEC0BF000C157F5C2
:103E500001C158F502C159F503C15AF500C15BF51E
:103E600001C15CF502C15DF503C15EF5ADEF1FF068
:103E700004014D0E826F96EC0EF0290E0C6E00C1FF
:103E80000BF04DEC0BF000C15FF500C160F5ADEF3C
:103E90001FF004014C0E826F96EC0EF00401540EDC
:103EA000826F96EC0EF004012C0E826F96EC0EF0F1
:103EB00084C32AF185C32BF186C32CF187C32DF16E
:103EC00088C32EF189C32FF18AC330F18BC331F13E
:103ED0008DC332F18EC333F1010163EC31F0DAECC2
:103EE00030F00101000E046F000E056F010E066F29
:103EF000000E076F11EC30F0210E0C6E00C10BF0BC
:103F00004DEC0BF0220E0C6E01C10BF04DEC0BF0E2
:103F1000230E0C6E02C10BF04DEC0BF0240E0C6E58
:103F200003C10BF04DEC0BF000C161F501C162F56E
:103F300002C163F503C164F5ADEF1FF004014C0E3F
:103F4000826F96EC0EF00401490E826F96EC0EF033
:103F500004012C0E826F96EC0EF0250E64EC0BF033
:103F6000E8CF00F1260E64EC0BF0E8CF01F1270E4C
:103F700064EC0BF0E8CF02F1280E64EC0BF0E8CF14
:103F800003F19EEC30F061EC2EF00401730E826FB1
:103F900096EC0EF004012C0E826F96EC0EF015ECF0
:103FA00031F0290E64EC0BF0E8CF00F19EEC30F01C
:103FB00061EC2EF004016D0E826F96EC0EF00401A0
:103FC0002C0E826F96EC0EF05BC500F15CC501F122
:103FD0005DC502F15EC503F19EEC30F061EC2EF0A0
:103FE0000401730E826F96EC0EF004012C0E826FAA
:103FF00096EC0EF015EC31F060C500F19EEC30F05F
:1040000061EC2EF004016D0E826F96EC0EF004014F
:104010002C0E826F96EC0EF061C500F162C501F1C5
:1040200063C502F164C503F133EC2AF004012C0EE0
:10403000826F96EC0EF0A0EC0EF018EF2AF083C31E
:104040002AF184C32BF185C32CF186C32DF187C3DC
:104050002EF188C32FF189C330F18AC331F18BC3AC
:1040600032F18CC333F1010163EC31F0DAEC30F062
:10407000160E0C6E00C10BF04DEC0BF0170E0C6E13
:1040800001C10BF04DEC0BF0180E0C6E02C10BF0E1
:104090004DEC0BF0190E0C6E03C10BF04DEC0BF058
:1040A00000C18EF101C18FF102C190F103C191F104
:1040B00000C192F101C193F102C194F103C195F1E4
:1040C00001EF21F083C32AF184C32BF185C32CF1C6
:1040D00086C32DF187C32EF188C32FF189C330F138
:1040E0008AC331F18BC332F18CC333F1010163EC2C
:1040F00031F0DAEC30F000C18EF101C18FF102C174
:1041000090F103C191F100C192F101C193F102C19B
:1041100094F103C195F101EF21F083C32AF184C327
:104120002BF185C32CF186C32DF187C32EF188C3F3
:104130002FF189C330F18AC331F18CC332F18DC3C1
:1041400033F1010163EC31F0DAEC30F00101000EE3
:10415000046F000E056F010E066F000E076F11EC65
:1041600030F01A0E0C6E00C10BF04DEC0BF01B0E74
:104170000C6E01C10BF04DEC0BF01C0E0C6E02C16D
:104180000BF04DEC0BF01D0E0C6E03C10BF04DEC63
:104190000BF000C196F101C197F102C198F103C182
:1041A00099F101EF21F083C32AF184C32BF185C378
:1041B0002CF186C32DF187C32EF188C32FF189C35B
:1041C00030F18AC331F18CC332F18DC333F1010177
:1041D00063EC31F0DAEC30F00101000E046F000EF8
:1041E000056F010E066F000E076F11EC30F000C175
:1041F00096F101C197F102C198F103C199F101EF64
:1042000021F0160E64EC0BF0E8CF00F1170E64EC11
:104210000BF0E8CF01F1180E64EC0BF0E8CF02F1DF
:10422000190E64EC0BF0E8CF03F19EEC30F061EC7A
:104230002EF00401730E826F96EC0EF004012C0E2A
:10424000826F96EC0EF08EC100F18FC101F190C12A
:1042500002F191C103F19EEC30F061EC2EF004010B
:10426000730E826F96EC0EF004012C0E826F96ECAA
:104270000EF01A0E64EC0BF0E8CF00F11B0E64ECAC
:104280000BF0E8CF01F11C0E64EC0BF0E8CF02F16B
:104290001D0E64EC0BF0E8CF03F133EC2AF00401BF
:1042A0002C0E826F96EC0EF096C100F197C101F1D1
:1042B00098C102F199C103F133EC2AF0A0EC0EF0A1
:1042C00018EF2AF00401690E826F96EC0EF00401DB
:1042D0002C0E826F96EC0EF00101040E006F000EA2
:1042E000016F000E026F000E036F9EEC30F02CC1C8
:1042F00082F40401300E822796EC0EF02DC182F478
:104300000401300E822796EC0EF02EC182F40401D7
:10431000300E822796EC0EF02FC182F40401300E8D
:10432000822796EC0EF030C182F40401300E822711
:1043300096EC0EF031C182F40401300E822796EC27
:104340000EF032C182F40401300E822796EC0EF09A
:1043500033C182F40401300E822796EC0EF0040182
:104360002C0E826F96EC0EF001010D0E006F000E08
:10437000016F000E026F000E036F9EEC30F02CC137
:1043800082F40401300E822796EC0EF02DC182F4E7
:104390000401300E822796EC0EF02EC182F4040147
:1043A000300E822796EC0EF02FC182F40401300EFD
:1043B000822796EC0EF030C182F40401300E822781
:1043C00096EC0EF031C182F40401300E822796EC97
:1043D0000EF032C182F40401300E822796EC0EF00A
:1043E00033C182F40401300E822796EC0EF00401F2
:1043F0002C0E826F96EC0EF00101490E006F000E3C
:10440000016F000E026F000E036F9EEC30F02CC1A6
:1044100082F40401300E822796EC0EF02DC182F456
:104420000401300E822796EC0EF02EC182F40401B6
:10443000300E822796EC0EF02FC182F40401300E6C
:10444000822796EC0EF030C182F40401300E8227F0
:1044500096EC0EF031C182F40401300E822796EC06
:104460000EF032C182F40401300E822796EC0EF079
:1044700033C182F40401300E822796EC0EF0040161
:104480002C0E826F96EC0EF0200EF86EF76AF66A2C
:1044900004010900F5CF82F496EC0EF00900F5CF87
:1044A00082F496EC0EF00900F5CF82F496EC0EF053
:1044B0000900F5CF82F496EC0EF00900F5CF82F4F6
:1044C00096EC0EF00900F5CF82F496EC0EF00900A0
:1044D000F5CF82F496EC0EF00900F5CF82F496EC5D
:1044E0000EF0A0EC0EF018EF2AF08351630AD8A466
:1044F00016EF2AF08451610AD8A416EF2AF08551EC
:104500006C0AD8A416EF2AF08651410A3FE0865182
:10451000440A1BE08651420AD8B4D9EF22F08651F2
:10452000350AD8B4A2EF2BF08651360AD8B4F7EF8B
:104530002BF08651370AD8B460EF2CF08651380A38
:10454000D8B4BEEF2CF016EF2AF00798079A0401B2
:104550007A0E826F96EC0EF00401780E826F96EC64
:104560000EF00401640E826F96EC0EF00401550EFD
:10457000826F96EC0EF0C2EF22F004014C0E826FB7
:1045800096EC0EF0A0EC0EF018EF2AF00788079AD0
:1045900004017A0E826F96EC0EF00401410E826FD8
:1045A00096EC0EF00401610E826F96EC0EF0B6EF01
:1045B00022F00798078A04017A0E826F96EC0EF0BB
:1045C0000401420E826F96EC0EF00401610E826FC0
:1045D00096EC0EF0B6EF22F001016667F7EF22F0DD
:1045E0006767F7EF22F06867F7EF22F0696716D088
:1045F00001014F6703EF23F0506703EF23F051678A
:1046000003EF23F052670AD00101000E006F000E85
:10461000016F000E026F000E036F120011B80AD076
:104620000101620E046F010E056F000E066F000E91
:10463000076F09D00101A70E046F020E056F000E6F
:10464000066F000E076F66C100F167C101F168C116
:1046500002F169C103F100EC30F003BFA0EF23F0D9
:10466000119A119C0101000E046FA80E056F550EE2
:10467000066F020E076F66C100F167C101F168C1E4
:1046800002F169C103F166C18AF167C18BF168C1AA
:104690008CF169C18DF100EC30F003BF0BD001014A
:1046A000000E8A6FA80E8B6F550E8C6F020E8D6FE9
:1046B000118A119C0E0E64EC0BF0E8CF18F10F0E6E
:1046C00064EC0BF0E8CF19F1100E64EC0BF0E8CFBE
:1046D0001AF1110E64EC0BF0E8CF1BF149EC2FF04E
:1046E0008AC104F18BC105F18CC106F18DC107F1BE
:1046F00000EC30F007820DEC2FF049EC2FF0079220
:104700000DEC2FF08AC100F18BC101F18CC102F1D7
:104710008DC103F107920DEC2FF0CC0E046FE00E6B
:10472000056F870E066F050E076F00EC30F000C1B5
:1047300018F101C119F102C11AF103C11BF140D0F6
:1047400013AAA5EF23F0138E139A119C119A01015D
:10475000800E006F1A0E016F060E026F000E036FBF
:104760004FC104F150C105F151C106F152C107F129
:1047700000EC30F003AF05D015EC31F0118C119A3C
:1047800012000E0E64EC0BF0E8CF18F10F0E64EC83
:104790000BF0E8CF19F1100E64EC0BF0E8CF1AF132
:1047A000110E64EC0BF0E8CF1BF14FC100F150C1CA
:1047B00001F151C102F152C103F107820DEC2FF05A
:1047C00018C100F119C101F11AC102F11BC103F1B5
:1047D00012000784BAC166F1BBC167F1BCC168F1C0
:1047E000BDC169F14BC14FF14CC150F14DC151F107
:1047F0004EC152F157C159F158C15AF10794010104
:1048000066670AEF24F067670AEF24F068670AEF2B
:1048100024F0696716D001014F6716EF24F0506746
:1048200016EF24F0516716EF24F052670AD0010109
:10483000000E006F000E016F000E026F000E036F7E
:10484000120011B80AD00101620E046F010E056F4B
:10485000000E066F000E076F09D00101A70E046F4E
:10486000020E056F000E066F000E076F66C100F1A5
:1048700067C101F168C102F169C103F100EC30F0D8
:1048800003BFA2EF24F00101000E046FA80E056F14
:10489000550E066F020E076F66C100F167C101F188
:1048A00068C102F169C103F166C18AF167C18BF188
:1048B00068C18CF169C18DF100EC30F003BF09D003
:1048C0000101000E8A6FA80E8B6F550E8C6F020EC1
:1048D0008D6F49EC2FF000C104F101C105F102C157
:1048E00006F103C107F1000E006FA00E016F980ED4
:1048F000026F7B0E036F31EC30F000C118F101C183
:1049000019F102C11AF103C11BF1000E006FA00ED4
:10491000016F980E026F7B0E036F8AC104F18BC189
:1049200005F18CC106F18DC107F131EC30F018C1F1
:1049300004F119C105F11AC106F11BC107F100EC20
:1049400030F012000101A80E006F610E016F000E21
:10495000026F000E036F4FC104F150C105F151C148
:1049600006F152C107F100EC30F003AF0AD00101AB
:10497000A80E006F610E016F000E026F000E036F34
:1049800000D0C80E006FAF0E016F000E026F000E58
:10499000036F4FC104F150C105F151C106F152C17D
:1049A00007F111EC30F012000401730E826F96ECE7
:1049B0000EF004012C0E826F96EC0EF0078462C19B
:1049C00066F163C167F164C168F165C169F14BC10A
:1049D0004FF14CC150F14DC151F14EC152F157C18F
:1049E00059F158C15AF10794FAEC24F0A0EC0EF0FA
:1049F00018EF2AF066C100F167C101F168C102F148
:104A000069C103F101019EEC30F061EC2EF004016C
:104A1000630E826F96EC0EF004012C0E826F96EC02
:104A20000EF04FC100F150C101F151C102F152C16C
:104A300003F101019EEC30F061EC2EF00401660EF2
:104A4000826F96EC0EF004012C0E826F96EC0EF045
:104A500015EC31F059C100F15AC101F101019EEC90
:104A600030F061EC2EF00401740E826F96EC0EF0C3
:104A7000120010820401530E826F96EC0EF00401B6
:104A80002C0E826F96EC0EF083C32AF184C32BF1B7
:104A900085C32CF186C32DF187C32EF188C32FF176
:104AA00089C330F18AC331F18BC332F18CC333F146
:104AB000010163EC31F0DAEC30F000C166F101C1C4
:104AC00067F102C168F103C169F18EC32AF18FC396
:104AD0002BF190C32CF191C32DF192C32EF193C30E
:104AE0002FF194C330F195C331F196C332F197C3DE
:104AF00033F1010163EC31F0DAEC30F000C14FF139
:104B000001C150F102C151F103C152F156EC31F033
:104B100099C32FF19AC330F19BC331F19CC332F199
:104B20009DC333F1010163EC31F0DAEC30F000C1E8
:104B300059F101C15AF1FAEC24F004012C0E826FF4
:104B400096EC0EF0B4EF25F0118E1CA002D01CAE36
:104B5000108C1BBE02D01BA4108E03018251520A7E
:104B600002E10F8201D00F928251750A02E1108496
:104B700001D010948251550A02E1108601D010969E
:104B80008351310A03E11382138402D013921394E8
:104B900003018351660A01E056D00401660E826F5C
:104BA00096EC0EF004012C0E826F96EC0EF0E9EC00
:104BB00023F09EEC30F02AC182F40401300E8227EB
:104BC00096EC0EF02BC182F40401300E822796EC95
:104BD0000EF02CC182F40401300E822796EC0EF008
:104BE0002DC182F40401300E822796EC0EF02EC106
:104BF00082F40401300E822796EC0EF02FC182F46D
:104C00000401300E822796EC0EF030C182F40401CC
:104C1000300E822796EC0EF031C182F40401300E82
:104C2000822796EC0EF032C182F40401300E822706
:104C300096EC0EF033C182F40401300E822796EC1C
:104C40000EF016EF2AF011A003D011A401D01084A9
:104C5000078410B28DEF26F010A471EF26F0BAC1D0
:104C600066F1BBC167F1BCC168F1BDC169F1BEC1EC
:104C70006AF1BFC16BF1C0C16CF1C1C16DF1C2C1BC
:104C80006EF1C3C16FF1C4C170F1C5C171F1C6C18C
:104C900072F1C7C173F1C8C174F1C9C175F1CAC15C
:104CA00076F1CBC177F1CCC178F1CDC179F1CEC12C
:104CB0007AF1CFC17BF1D0C17CF1D1C17DF1D2C1FC
:104CC0007EF1D3C17FF1D4C180F1D5C181F1D6C1CC
:104CD00082F1D7C183F1D8C184F1D9C185F179EFCF
:104CE00026F062C166F163C167F164C168F165C114
:104CF00069F1BAC186F1BBC187F1BCC188F1BDC100
:104D000089F14BC14FF14CC150F14DC151F14EC130
:104D100052F157C159F158C15AF107940FA0AFEFA2
:104D200026F0010196679CEF26F097679CEF26F02E
:104D300098679CEF26F09967A0EF26F0AFEF26F07A
:104D4000ECEC22F096C104F197C105F198C106F18F
:104D500099C107F100EC30F003BFDCEF29F0ECEC77
:104D600022F00101000E046F000E056F010E066FA8
:104D7000000E076F31EC30F011A02AD011A228D01C
:104D80009EEC30F0296701D005D004012D0E826F12
:104D900096EC0EF030C182F40401300E822796ECBE
:104DA0000EF031C182F40401300E822796EC0EF031
:104DB00032C182F40401300E822796EC0EF033C12A
:104DC00082F40401300E822796EC0EF0A0EC0EF077
:104DD00012A8C5D012981DC01EF01E3A1E42070E22
:104DE0001E1600011E50000AD8B47BEF27F0000108
:104DF0001E50010AD8B407EF27F000011E50020A26
:104E0000D8B405EF27F0ADEF27F0ADEF27F015ECA4
:104E100031F02DC001F12EC000F1D89001330033E4
:104E2000D890013300330101630E046F000E056F4B
:104E3000000E066F000E076F31EC30F0280E046F85
:104E4000000E056F000E066F000E076F00EC30F0CD
:104E500000C130F015EC31F02BC001F1019F019D34
:104E60002CC000F10101A40E046F000E056F000EAE
:104E7000066F000E076F31EC30F000C12FF000C15B
:104E800004F101C105F102C106F103C107F1640E8D
:104E9000006F000E016F000E026F000E036F00EC3A
:104EA00030F0050E046F000E056F000E066F000E49
:104EB000076F31EC30F000C104F101C105F102C10E
:104EC00006F103C107F115EC31F030C000F100EC40
:104ED00030F000C131F031C0E8FF050F305C03E76E
:104EE0008A84ADEF27F031C0E8FF0A0F305C01E69D
:104EF0008A94ADEF27F000C124F101C125F102C170
:104F000026F103C127F115EC31F01BEC31F01D50F7
:104F10001F0BE8CF00F10101640E046F000E056F56
:104F2000000E066F000E076F11EC30F024C104F183
:104F300025C105F126C106F127C107F100EC30F0CB
:104F400003BF02D08A9401D08A8424C100F125C114
:104F500001F126C102F127C103F118EF2AF000C1C7
:104F600024F101C125F102C126F103C127F110AEE0
:104F70004DD0109E00C108F101C109F102C10AF132
:104F800003C10BF19EEC30F030C1E2F131C1E3F12D
:104F900032C1E4F133C1E5F108C100F109C101F109
:104FA0000AC102F10BC103F101016C0E046F070E7F
:104FB000056F000E066F000E076F00EC30F003BFA8
:104FC00004D00101550EE66F1CD008C100F109C1E3
:104FD00001F10AC102F10BC103F10101A40E046F3A
:104FE000060E056F000E066F000E076F00EC30F026
:104FF00003BF04D001017F0EE66F03D00101FF0E55
:10500000E66F1F8E11AEDCEF29F0119E24C100F176
:1050100025C101F126C102F127C103F111A005D07C
:1050200011A203D00FB0DCEF29F010A41FEF28F07D
:105030000401750E826F96EC0EF024EF28F0040147
:10504000720E826F96EC0EF004012C0E826F96ECBD
:105050000EF09EEC30F0296733EF28F00401200EAB
:10506000826F36EF28F004012D0E826F96EC0EF061
:1050700030C182F40401300E822796EC0EF031C16B
:1050800082F40401300E822796EC0EF004012E0EFD
:10509000826F96EC0EF032C182F40401300E82274A
:1050A00096EC0EF033C182F40401300E822796ECA8
:1050B0000EF004016D0E826F96EC0EF004012C0EC2
:1050C000826F96EC0EF04FC100F150C101F151C159
:1050D00002F152C103F101019EEC30F061EC2EF0BF
:1050E0000401480E826F96EC0EF004017A0E826F76
:1050F00096EC0EF004012C0E826F96EC0EF066C159
:1051000000F167C101F168C102F169C103F1010158
:105110009EEC30F061EC2EF00401630E826F96EC91
:105120000EF004012C0E826F96EC0EF066C100F1B9
:1051300067C101F168C102F169C103F101010A0E01
:10514000046F000E056F000E066F000E076F11EC66
:1051500030F0000E046F120E056F000E066F000E89
:10516000076F31EC30F09EEC30F02AC182F404017C
:10517000300E822796EC0EF02BC182F40401300E23
:10518000822796EC0EF02CC182F40401300E8227A7
:1051900096EC0EF02DC182F40401300E822796ECBD
:1051A0000EF02EC182F40401300E822796EC0EF030
:1051B0002FC182F40401300E822796EC0EF030C12C
:1051C00082F40401300E822796EC0EF004012E0EBC
:1051D000826F96EC0EF031C182F40401300E82270A
:1051E00096EC0EF032C182F40401300E822796EC68
:1051F0000EF033C182F40401300E822796EC0EF0DB
:105200000401730E826F96EC0EF004012C0E826F77
:1052100096EC0EF015EC31F059C100F15AC101F1D4
:1052200042EC2BF013A264EF29F004012C0E826FE4
:1052300096EC0EF086C166F187C167F188C168F10E
:1052400089C169F1ECEC22F00101000E046F000E3F
:10525000056F010E066F000E076F31EC30F09EEC0B
:1052600030F0296739EF29F00401200E826F3CEFFE
:1052700029F004012D0E826F96EC0EF030C182F4FD
:105280000401300E822796EC0EF031C182F4040145
:10529000300E822796EC0EF004012E0E826F96ECF3
:1052A0000EF032C182F40401300E822796EC0EF02B
:1052B00033C182F40401300E822796EC0EF0040113
:1052C0006D0E826F96EC0EF013A48BEF29F00401A3
:1052D0002C0E826F96EC0EF013AC79EF29F00401DE
:1052E000500E826F96EC0EF0139C1398139A8BEF6E
:1052F00029F013AE86EF29F00401460E826F96EC7A
:105300000EF0139E1398139A8BEF29F00401530E9D
:10531000826F96EC0EF037B0A2EF29F004012C0E4C
:10532000826F96EC0EF08BB09DEF29F00401440ED5
:10533000826F96EC0EF0A2EF29F00401530E826FFB
:1053400096EC0EF00FB2A8EF29F00FA0DAEF29F0DB
:1053500004012C0E826F96EC0EF0200EF86EF76AA8
:10536000F66A04010900F5CF82F496EC0EF009000C
:10537000F5CF82F496EC0EF00900F5CF82F496ECAE
:105380000EF00900F5CF82F496EC0EF00900F5CF8F
:1053900082F496EC0EF00900F5CF82F496EC0EF054
:1053A0000900F5CF82F496EC0EF00900F5CF82F4F7
:1053B00096EC0EF0A0EC0EF00F90109E129818EFE5
:1053C0002AF00401630E826F96EC0EF004012C0E9D
:1053D000826F96EC0EF01EEC2AF004012C0E826F08
:1053E00096EC0EF091EC2AF004012C0E826F96ECF4
:1053F0000EF00DEC2BF004012C0E826F96EC0EF0EB
:105400000101F80E006FCD0E016F660E026F030EE4
:10541000036F33EC2AF004012C0E826F96EC0EF031
:1054200023EC2BF0A0EC0EF018EF2AF0A0EC0EF01D
:105430000301C26B0790109227EF2DF0D8900E0E4B
:1054400064EC0BF0E8CF00F10F0E64EC0BF0E8CF4A
:1054500001F1100E64EC0BF0E8CF02F1110E64ECD8
:105460000BF0E8CF03F10101000E046F000E056F91
:10547000010E066F000E076F31EC30F09EEC30F03D
:105480002AC182F40401300E822796EC0EF02BC163
:1054900082F40401300E822796EC0EF02CC182F4C7
:1054A0000401300E822796EC0EF02DC182F4040127
:1054B000300E822796EC0EF02EC182F40401300EDD
:1054C000822796EC0EF02FC182F40401300E822761
:1054D00096EC0EF030C182F40401300E822796EC77
:1054E0000EF031C182F40401300E822796EC0EF0EA
:1054F00004012E0E826F96EC0EF032C182F404018C
:10550000300E822796EC0EF033C182F40401300E87
:10551000822796EC0EF004016D0E826F96EC0EF071
:105520001200120E64EC0BF0E8CF00F1130E64ECE5
:105530000BF0E8CF01F1140E64EC0BF0E8CF02F1B0
:10554000150E64EC0BF0E8CF03F101010A0E046FB5
:10555000000E056F000E066F000E076F11EC30F0A5
:10556000000E046F120E056F000E066F000E076F1F
:1055700031EC30F09EEC30F02AC182F40401300EA0
:10558000822796EC0EF02BC182F40401300E8227A4
:1055900096EC0EF02CC182F40401300E822796ECBA
:1055A0000EF02DC182F40401300E822796EC0EF02D
:1055B0002EC182F40401300E822796EC0EF02FC12A
:1055C00082F40401300E822796EC0EF030C182F492
:1055D0000401300E822796EC0EF004012E0E826F2D
:1055E00096EC0EF031C182F40401300E822796EC65
:1055F0000EF032C182F40401300E822796EC0EF0D8
:1056000033C182F40401300E822796EC0EF00401BF
:10561000730E826F96EC0EF012000A0E64EC0BF023
:10562000E8CF00F10B0E64EC0BF0E8CF01F10C0EAB
:1056300064EC0BF0E8CF02F10D0E64EC0BF0E8CF58
:1056400003F142EF2BF0060E64EC0BF0E8CF00F113
:10565000070E64EC0BF0E8CF01F1080E64EC0BF0E0
:10566000E8CF02F1090E64EC0BF0E8CF03F142EF52
:105670002BF0010115EC31F0078457C100F158C13E
:1056800001F107940101E80E046F800E056F000E12
:10569000066F000E076F11EC30F0000E046F040E61
:1056A000056F000E066F000E076F31EC30F0880EAC
:1056B000046F130E056F000E066F000E076F00ECEF
:1056C00030F00A0E046F000E056F000E066F000E1C
:1056D000076F31EC30F09EEC30F00101296776EF76
:1056E0002BF00401200E826F79EF2BF004012D0EB8
:1056F000826F96EC0EF030C182F40401300E8227E6
:1057000096EC0EF031C182F40401300E822796EC43
:105710000EF032C182F40401300E822796EC0EF0B6
:1057200004012E0E826F96EC0EF033C182F4040158
:10573000300E822796EC0EF00401430E826F96EC39
:105740000EF0120087C32AF188C32BF189C32CF114
:105750008AC32DF18BC32EF18CC32FF18DC330F191
:105760008EC331F190C332F191C333F10101296B42
:1057700063EC31F0DAEC30F00101000E046F000E42
:10578000056F010E066F000E076F11EC30F00E0E64
:105790000C6E00C10BF04DEC0BF00F0E0C6E01C146
:1057A0000BF04DEC0BF0100E0C6E02C10BF04DEC3B
:1057B0000BF0110E0C6E03C10BF04DEC0BF004015D
:1057C0007A0E826F96EC0EF004012C0E826F96EC2E
:1057D0000EF00401350E826F96EC0EF004012C0ED3
:1057E000826F96EC0EF01EEC2AF0C2EF22F087C317
:1057F0002AF188C32BF189C32CF18AC32DF18BC305
:105800002EF18CC32FF18DC330F18EC331F190C3D3
:1058100032F191C333F10101296B63EC31F0DAEC21
:1058200030F0880E046F130E056F000E066F000E29
:10583000076F05EC30F0000E046F040E056F000ECC
:10584000066F000E076F11EC30F00101E80E046FD7
:10585000800E056F000E066F000E076F31EC30F002
:105860000A0E0C6E00C10BF04DEC0BF00B0E0C6E23
:1058700001C10BF04DEC0BF00C0E0C6E02C10BF0E5
:105880004DEC0BF00D0E0C6E03C10BF04DEC0BF05C
:1058900004017A0E826F96EC0EF004012C0E826FDA
:1058A00096EC0EF00401360E826F96EC0EF00401B9
:1058B0002C0E826F96EC0EF00DEC2BF0C2EF22F066
:1058C00087C32AF188C32BF189C32CF18AC32DF138
:1058D0008BC32EF18CC32FF18DC330F18FC331F107
:1058E00090C332F191C333F1010163EC31F0DAEC92
:1058F00030F0000E046F120E056F000E066F000EE2
:10590000076F11EC30F001010A0E046F000E056FF5
:10591000000E066F000E076F31EC30F0120E0C6EA9
:1059200000C10BF04DEC0BF0130E0C6E01C10BF02F
:105930004DEC0BF0140E0C6E02C10BF04DEC0BF0A5
:10594000150E0C6E03C10BF04DEC0BF004017A0E3A
:10595000826F96EC0EF004012C0E826F96EC0EF026
:105960000401370E826F96EC0EF004012C0E826F4C
:1059700096EC0EF091EC2AF0C2EF22F087C32AF1E8
:1059800088C32BF189C32CF18AC32DF18BC32EF16F
:105990008CC32FF18DC330F18EC331F190C332F13E
:1059A00091C333F10101296B63EC31F0DAEC30F093
:1059B000880E046F130E056F000E066F000E076F42
:1059C00005EC30F0000E046F040E056F000E066F3C
:1059D000000E076F11EC30F00101E80E046F800E2D
:1059E000056F000E066F000E076F31EC30F0060EEB
:1059F0000C6E00C10BF04DEC0BF0070E0C6E01C1EC
:105A00000BF04DEC0BF0080E0C6E02C10BF04DECE0
:105A10000BF0090E0C6E03C10BF04DEC0BF0040102
:105A20007A0E826F96EC0EF004012C0E826F96ECCB
:105A30000EF00401380E826F96EC0EF004012C0E6D
:105A4000826F96EC0EF023EC2BF0C2EF22F007A849
:105A50009AEF2DF00101800E006F1A0E016F060EF5
:105A6000026F000E036F4BC104F14CC105F14DC133
:105A700006F14EC107F100EC30F003BFE0EF2DF06E
:105A80005BEC2EF04BC100F14CC101F14DC102F1B4
:105A90004EC103F107820DEC2FF018C104F119C1BA
:105AA00005F11AC106F11BC107F1F80E006FCD0E0A
:105AB000016F660E026F030E036F00EC30F00E0EE6
:105AC0000C6E00C10BF04DEC0BF00F0E0C6E01C113
:105AD0000BF04DEC0BF0100E0C6E02C10BF04DEC08
:105AE0000BF0110E0C6E03C10BF04DEC0BF00784A4
:105AF000010115EC31F057C100F158C101F10794D3
:105B00000A0E0C6E00C10BF04DEC0BF00B0E0C6E80
:105B100001C10BF04DEC0BF00C0E0C6E02C10BF042
:105B20004DEC0BF00D0E0C6E03C10BF04DEC0BF0B9
:105B3000E0EF2DF007AAE0EF2DF00784010115EC4E
:105B400031F057C100F158C101F10794060E0C6EF7
:105B500000C10BF04DEC0BF0070E0C6E01C10BF009
:105B60004DEC0BF0080E0C6E02C10BF04DEC0BF07F
:105B7000090E0C6E03C10BF04DEC0BF0078462C1F3
:105B800000F163C101F164C102F165C103F1079441
:105B9000120E0C6E00C10BF04DEC0BF0130E0C6EE0
:105BA00001C10BF04DEC0BF0140E0C6E02C10BF0AA
:105BB0004DEC0BF0150E0C6E03C10BF04DEC0BF021
:105BC0000798079A0401805181197F0B0DE09EA868
:105BD000FED714EE00F081517F0BE126E750812BB8
:105BE0000F01AD6EE2EF2DF005012F51000AD8B480
:105BF00023EF2EF081BA08EF2EF015B223EF2EF02E
:105C000005012F51010AD8B421EF2EF01AEF2EF022
:105C100005012F51000AD8B4DAEF38F005012F51F1
:105C2000010AD8B421EF2EF000011650050AD8B4AD
:105C3000DAEF38F081B823EF2EF05EEC32F05CEC56
:105C400033F073EC38F0C4EF0DF018C100F119C156
:105C500001F11AC102F11BC103F1000E046F000E25
:105C6000056F010E066F000E076F31EC30F029A1B1
:105C700050EF2EF02051D8B450EF2EF018C100F1A3
:105C800019C101F11AC102F11BC103F1000E046F29
:105C9000000E056F0A0E066F000E076F31EC30F034
:105CA00012000101045100130551011306510213A2
:105CB0000751031312000101186B196B1A6B1B6B50
:105CC00012002AC182F40401300E822796EC0EF0F5
:105CD0002BC182F40401300E822796EC0EF02CC109
:105CE00082F40401300E822796EC0EF02DC182F46E
:105CF0000401300E822796EC0EF02EC182F40401CE
:105D0000300E822796EC0EF02FC182F40401300E83
:105D1000822796EC0EF030C182F40401300E822707
:105D200096EC0EF031C182F40401300E822796EC1D
:105D30000EF032C182F40401300E822796EC0EF090
:105D400033C182F40401300E822796EC0EF012006B
:105D50002FC182F40401300E822796EC0EF030C180
:105D600082F40401300E822796EC0EF031C182F4E9
:105D70000401300E822796EC0EF032C182F4040149
:105D8000300E822796EC0EF033C182F40401300EFF
:105D9000822796EC0EF01200060E216E060E226E81
:105DA000060E236E212ED2EF2EF0222ED2EF2EF0F1
:105DB000232ED2EF2EF08B84020E216E020E226E65
:105DC000020E236E212EE2EF2EF0222EE2EF2EF0B5
:105DD000232EE2EF2EF08B941200FF0E226E22C0D3
:105DE00023F0030E216E8B84212EF3EF2EF0030E91
:105DF000216E232EF3EF2EF08B9422C023F0030E9E
:105E0000216E212E01EF2FF0030E216E233E01EFB4
:105E10002FF0222EEFEF2EF012000101005305E1CA
:105E2000015303E1025301E1002BD0EC2FF015ECFC
:105E300031F03951006F3A51016F420E046F4B0E31
:105E4000056F000E066F000E076F11EC30F000C1F9
:105E500004F101C105F102C106F103C107F118C146
:105E600000F119C101F11AC102F11BC103F107B21E
:105E70003EEF2FF005EC30F040EF2FF000EC30F06B
:105E800000C118F101C119F102C11AF103C11BF1DE
:105E9000120015EC31F059C100F15AC101F1060EA2
:105EA00064EC0BF0E8CF04F1070E64EC0BF0E8CFE4
:105EB00005F1080E64EC0BF0E8CF06F1090E64EC76
:105EC0000BF0E8CF07F100EC30F000C124F101C184
:105ED00025F102C126F103C127F1290E046F000E3E
:105EE000056F000E066F000E076F11EC30F0EE0E1E
:105EF000046F430E056F000E066F000E076F05EC72
:105F000030F024C104F125C105F126C106F127C1F5
:105F100007F111EC30F000C11CF101C11DF102C10B
:105F20001EF103C11FF1120E64EC0BF0E8CF04F177
:105F3000130E64EC0BF0E8CF05F1140E64EC0BF0DB
:105F4000E8CF06F1150E64EC0BF0E8CF07F10D0E6B
:105F5000006F000E016F000E026F000E036F11EC58
:105F600030F0180E046F000E056F000E066F000E65
:105F7000076F31EC30F01CC104F11DC105F11EC1E9
:105F800006F11FC107F105EC30F06A0E046F2A0E0E
:105F9000056F000E066F000E076F00EC30F0120068
:105FA000BF0EFA6E200E3A6F396BD890003701376A
:105FB00002370337D8B0E1EF2FF03A2FD6EF2FF0AA
:105FC00039073A070353D8B412000331070B80098D
:105FD0003F6F03390F0B010F396F80EC5FF0406F9B
:105FE000390580EC5FF0405D405F396B3F33D8B0DE
:105FF000392739333FA9F6EF2FF0405139271200E6
:1060000001013AEC31F0D8B0120001010351071937
:10601000346FFDEC30F0D8900751031934AF800F86
:1060200012000101346B21EC31F0D8A037EC31F0D3
:10603000D8B012000CEC31F015EC31F01F0E366FB9
:106040004DEC31F00B35D8B0FDEC30F0D8A0033575
:10605000D8B01200362F20EF30F034B124EC31F0FC
:1060600012000101346B04510511061107110008DB
:10607000D8A021EC31F0D8A037EC31F0D8B0120024
:10608000086B096B0A6B0B6B4DEC31F01F0E366F12
:106090004DEC31F007510B5DD8A45BEF30F00651A9
:1060A0000A5DD8A45BEF30F00551095DD8A45BEF21
:1060B00030F00451085DD8A06EEF30F00451085F55
:1060C0000551D8A0053D095F0651D8A0063D0A5FDD
:1060D0000751D8A0073D0B5FD8900081362F48EFBD
:1060E00030F034B124EC31F0346B21EC31F0D89045
:1060F00051EC31F007510B5DD8A48BEF30F0065115
:106100000A5DD8A48BEF30F00551095DD8A48BEF60
:1061100030F00451085DD8A09AEF30F0003F9AEFBC
:1061200030F0013F9AEF30F0023F9AEF30F0032B4E
:10613000D8B4120034B124EC31F012000101346BF8
:1061400021EC31F0D8B0120056EC31F0200E366F51
:10615000003701370237033711EE33F00A0E376F7D
:10616000E7360A0EE75CD8B0E76EE552372FB0EF9E
:1061700030F0362FA8EF30F034B12981D8901200DA
:1061800056EC31F0200E366F0037013702370337F7
:1061900011EE33F00A0E376FE7360A0EE75CD8B01F
:1061A000E76EE552372FCCEF30F0362FC4EF30F0EA
:1061B000D890120001010A0E346F200E366F11EED6
:1061C00029F03451376F0A0ED890E652D8B0E7263E
:1061D000E732372FE5EF30F003330233013300337A
:1061E000362FDFEF30F0E750FF0FD8A00335D8B0DF
:1061F000120029B124EC31F012000451002705519E
:10620000D8B0053D01270651D8B0063D02270751F9
:10621000D8B0073D032712000051086F0151096FE4
:1062200002510A6F03510B6F12000101006B016BE9
:10623000026B036B12000101046B056B066B076BAD
:1062400012000335D8A012000351800B001F011F5C
:10625000021F031F003F34EF31F0013F34EF31F0F4
:10626000023F34EF31F0032B342B032512000735A6
:10627000D8A012000751800B041F051F061F071F1F
:10628000043F4AEF31F0053F4AEF31F0063F4AEF55
:1062900031F0072B342B0725120000370137023766
:1062A0000337083709370A370B3712000101296B0A
:1062B0002A6B2B6B2C6B2D6B2E6B2F6B306B316B1A
:1062C000326B336B120001012A510F0B2A6F2B51D5
:1062D0000F0B2B6F2C510F0B2C6F2D510F0B2D6FA4
:1062E0002E510F0B2E6F2F510F0B2F6F30510F0BA5
:1062F000306F31510F0B316F32510F0B326F335101
:106300000F0B336F120000C124F101C125F102C14E
:1063100026F103C127F104C100F105C101F106C155
:1063200002F107C103F124C104F125C105F126C121
:1063300006F127C107F1120010A806D08994000EBB
:10634000C76E220EC66E05D08984000EC76E220E5F
:10635000C66E050EE82EFED7120010A802D0898462
:1063600001D08994050EE82EFED712009CEC31F086
:106370009E96C69E000EC96EFF0E9EB602D0E82EF7
:10638000FCD79E96C69E000EC96EFF0E9EB602D02A
:10639000E82EFCD7C9CFAFF59E96C69E000EC96EFB
:1063A000FF0E9EB602D0E82EFCD7C9CFB0F59E9660
:1063B000C69E000EC96EFF0E9EB602D0E82EFCD718
:1063C000C9CFB1F59E96C69E000EC96EFF0E9EB651
:1063D00002D0E82EFCD7C9CFB2F59E96C69E000E1D
:1063E000C96EFF0E9EB602D0E82EFCD7C9CFB3F51A
:1063F0009E96C69E000EC96EFF0E9EB602D0E82E77
:10640000FCD7C9CFB4F59E96C69E000EC96EFF0E8E
:106410009EB602D0E82EFCD7C9CFB5F5ADEC31F071
:1064200012009CEC31F09E96C69E800EC96EFF0E47
:106430009EB602D0E82EFCD79E96C69EAFC5C9FF79
:10644000FF0E9EB602D0E82EFCD79E96C69EB0C523
:10645000C9FFFF0E9EB602D0E82EFCD79E96C69EC0
:10646000B1C5C9FFFF0E9EB602D0E82EFCD79E969E
:10647000C69EB2C5C9FFFF0E9EB602D0E82EFCD75D
:106480009E96C69EB3C5C9FFFF0E9EB602D0E82EEB
:10649000FCD79E96C69EB4C5C9FFFF0E9EB602D01D
:1064A000E82EFCD79E96C69EB5C5C9FFFF0E9EB6C8
:1064B00002D0E82EFCD7ADEC31F012009CEC31F0AC
:1064C0009E96C69E070EC96EFF0E9EB602D0E82E9F
:1064D000FCD79E96C69E000EC96EFF0E9EB602D0D9
:1064E000E82EFCD7C9CFAFF59E96C69E000EC96EAA
:1064F000FF0E9EB602D0E82EFCD7C9CFB0F59E960F
:10650000C69E000EC96EFF0E9EB602D0E82EFCD7C6
:10651000C9CFB1F59E96C69E000EC96EFF0E9EB6FF
:1065200002D0E82EFCD7C9CFB2F5ADEC31F09CEC2F
:1065300031F09E96C69E25C0C9FFFF0E9EB602D0C2
:10654000E82EFCD79E96C69E000EC96EFF0E9EB624
:1065500002D0E82EFCD7C9CFB6F5ADEC31F0120071
:106560009CEC31F09E96C69E870EC96EFF0E9EB6BD
:1065700002D0E82EFCD79E96C69EAFC5C9FFFF0E7F
:106580009EB602D0E82EFCD79E96C69EB0C5C9FF27
:10659000FF0E9EB602D0E82EFCD79E96C69EB1C5D1
:1065A000C9FFFF0E9EB602D0E82EFCD79E96C69E6F
:1065B000B2C5C9FFFF0E9EB602D0E82EFCD7ADECE7
:1065C00031F09CEC31F09E96C69E26C0C9FFFF0EAE
:1065D0009EB602D0E82EFCD79E96C69EB6C5C9FFD1
:1065E000FF0E9EB602D0E82EFCD7ADEC31F01200C3
:1065F0009CEC31F09E96C69E870EC96EFF0E9EB62D
:1066000002D0E82EFCD79E96C69E000EC96EFF0EE5
:106610009EB602D0E82EFCD79E96C69E800EC96E0E
:10662000FF0E9EB602D0E82EFCD79E96C69E800E28
:10663000C96EFF0E9EB602D0E82EFCD79E96C69E6F
:10664000800EC96EFF0E9EB602D0E82EFCD7ADECD0
:1066500031F012009CEC31F09E96C69E870EC96EFA
:10666000FF0E9EB602D0E82EFCD79E96C69E000E68
:10667000C96EFF0E9EB602D0E82EFCD79E96C69E2F
:10668000000EC96EFF0E9EB602D0E82EFCD79E9675
:10669000C69E800EC96EFF0E9EB602D0E82EFCD7B5
:1066A0009E96C69E800EC96EFF0E9EB602D0E82E44
:1066B000FCD7ADEC31F0120010A817D09CEC31F0F3
:1066C0009E96C69E8F0EC96EFF0E9EB602D0E82E15
:1066D000FCD79E96C69E000EC96EFF0E9EB602D0D7
:1066E000E82EFCD7ADEC31F012005EEC32F0120077
:1066F00010A82DD09CEC31F09E96C69E26C0C9FFF6
:10670000FF0E9EB602D0E82EFCD79E96C69E450E82
:10671000C96EFF0E9EB602D0E82EFCD7ADEC31F06C
:106720009CEC31F09E96C69E8F0EC96EFF0E9EB6F3
:1067300002D0E82EFCD79E96C69E000EC96EFF0EB4
:106740009EB602D0E82EFCD7ADEC31F012009CECE6
:1067500031F09E96C69E26C0C9FFFF0E9EB602D09F
:10676000E82EFCD79E96C69E010EC96EFF0E9EB601
:1067700002D0E82EFCD7ADEC31F09CEC31F09E96C7
:10678000C69E910EC96EFF0E9EB602D0E82EFCD7B3
:106790009E96C69EA50EC96EFF0E9EB602D0E82E2E
:1067A000FCD7ADEC31F012009CEC31F09E96C69E09
:1067B00026C0C9FFFF0E9EB602D0E82EFCD79E96DB
:1067C000C69E810EC96EFF0E9EB602D0E82EFCD783
:1067D000ADEC31F012009CEC31F09E96C69E26C0C6
:1067E000C9FFFF0E9EB602D0E82EFCD79E96C69E2D
:1067F000010EC96EFF0E9EB602D0E82EFCD7ADEC9E
:1068000031F012009CEC31F09E96C69E910EC96E3E
:10681000FF0E9EB602D0E82EFCD79E96C69EA50E11
:10682000C96EFF0E9EB602D0E82EFCD7ADEC31F05B
:1068300012009CEC31F09E96C69E910EC96EFF0E22
:106840009EB602D0E82EFCD79E96C69E000EC96E5C
:10685000FF0E9EB602D0E82EFCD7ADEC31F0120050
:106860000501256B266B276B286B899A400EC76E36
:10687000200EC66E9E96C69E030EC96EFF0E9EB675
:1068800002D0E82EFCD79E96C69E27C5C9FFFF0EF4
:106890009EB602D0E82EFCD79E96C69E26C5C9FF9E
:1068A000FF0E9EB602D0E82EFCD79E96C69E25C54A
:1068B000C9FFFF0E9EB602D0E82EFCD79E96C69E5C
:1068C000C952FF0E9EB602D0E82EFCD7898A0F016E
:1068D000C950FF0A01E1120005012E51130A05E01B
:1068E00005012E51170A0CE012000501E00E256F7C
:1068F000FF0E266F0F0E276F000E286F89EF34F002
:106900000501E00E256FFF0E266FFF0E276F000EAC
:10691000286F899A400EC76E200EC66E9E96C69E40
:10692000030EC96EFF0E9EB602D0E82EFCD79E96CF
:10693000C69E27C5C9FFFF0E9EB602D0E82EFCD723
:106940009E96C69E26C5C9FFFF0E9EB602D0E82EB3
:10695000FCD79E96C69E25C5C9FFFF0E9EB602D0E7
:10696000E82EFCD79E96C69EC952FF0E9EB602D058
:10697000E82EFCD7898A0F01C950FF0A1DE00501E6
:106980002E51130A05E005012E51170A0BE01200E3
:106990000501000E256F000E266F100E276F000EEA
:1069A000286F12000501000E256F000E266F000EE5
:1069B000276F010E286F12000501256B266B276BD0
:1069C000286B05012E51130A05E005012E51170A07
:1069D0000CE012000501000E216F000E226F080E60
:1069E000236F000E246FFEEF34F00501000E216FBF
:1069F000000E226F800E236F000E246F21C500F160
:106A000022C501F123C502F124C503F125C504F116
:106A100026C505F127C506F128C507F151EC2EF072
:106A200000C125F501C126F502C127F503C128F5EE
:106A3000899A400EC76E200EC66E9E96C69E030EA5
:106A4000C96EFF0E9EB602D0E82EFCD79E96C69E5B
:106A500027C5C9FFFF0E9EB602D0E82EFCD79E9632
:106A6000C69E26C5C9FFFF0E9EB602D0E82EFCD7F3
:106A70009E96C69E25C5C9FFFF0E9EB602D0E82E83
:106A8000FCD79E96C69EC952FF0E9EB602D0E82E37
:106A9000FCD7898AC950FF0A08E104C125F505C160
:106AA00026F506C127F507C128F5D890050124333E
:106AB0002333223321332151E00B216F050121675C
:106AC00069EF35F0226769EF35F0236769EF35F03C
:106AD0002467FEEF34F00501200E2527E86A2623FF
:106AE000E86A2723E86A28231200E86A05012E5184
:106AF000130A06E005012E51170A0BE0020E1200E0
:106B000005012851000A03E12751F00B07E0010EAF
:106B1000120005012851000A01E0010E120029C5EA
:106B200000F12AC501F12BC502F12CC503F125C5E1
:106B300004F126C505F127C506F128C507F100ECCB
:106B400030F003BF120075EC35F0D8A407EF36F033
:106B5000899A400EC76E200EC66E9E96C69E060E81
:106B6000C96EFF0E9EB602D0E82EFCD7898A899A9C
:106B70009E96C69E020EC96EFF0E9EB602D0E82EED
:106B8000FCD79E96C69E27C5C9FFFF0E9EB602D0B3
:106B9000E82EFCD79E96C69E26C5C9FFFF0E9EB660
:106BA00002D0E82EFCD79E96C69E25C5C9FFFF0ED3
:106BB0009EB602D0E82EFCD79E96C69E000EC96EE9
:106BC000FF0E9EB602D0E82EFCD7898A899A9E963F
:106BD000C69E050EC96EFF0E9EB602D0E82EFCD7EB
:106BE0009E96C69EC952FF0E9EB602D0E82EFCD7D6
:106BF000C9B0F0EF35F0898A0501200E2527E86A33
:106C00002623E86A2723E86A28238FEF35F012004D
:106C1000899A400EC76E200EC66E9E96C69E060EC0
:106C2000C96EFF0E9EB602D0E82EFCD7898A899ADB
:106C30009E96C69EC70EC96EFF0E9EB602D0E82E67
:106C4000FCD7898A0501256B266B276B286B120000
:106C5000899A400EC76E200EC66E9E96C69E050E81
:106C6000C96EFF0E9EB602D0E82EFCD79E96C69E39
:106C7000C952FF0E9EB602D0E82EFCD7C9CF37F519
:106C8000898A1200899A400EC76E200EC66E9E96A3
:106C9000C69EB90EC96EFF0E9EB602D0E82EFCD776
:106CA000898A1200899A400EC76E200EC66E9E9683
:106CB000C69EAB0EC96EFF0E9EB602D0E82EFCD764
:106CC000898AFF0EE82EFED7120075EC35F0D8A4A5
:106CD0001200899A400EC76E200EC66E9E96C69E02
:106CE000030EC96EFF0E9EB602D0E82EFCD79E960C
:106CF000C69E27C5C9FFFF0E9EB602D0E82EFCD760
:106D00009E96C69E26C5C9FFFF0E9EB602D0E82EEF
:106D1000FCD79E96C69E25C5C9FFFF0E9EB602D023
:106D2000E82EFCD79E96C69EC952FF0E9EB602D094
:106D3000E82EFCD7898A0F01C950FF0AD8A4E4EFD6
:106D400037F00501FE0E376F0501FF0E536FFF0E82
:106D5000546FFF0E556FFF0E566F15A637991586A7
:106D6000B6EC31F0AFC538F5B0C539F5B1C53AF577
:106D7000B2C53BF5B3C53CF5B4C53DF5B5C53EF56B
:106D80000784BAC166F1BBC167F1BCC168F1BDC17E
:106D900069F14BC14FF14CC150F14DC151F14EC1A0
:106DA00052F157C159F158C15AF100011650010A68
:106DB000D8B4E9EF36F000011650020AD8B40EEF4D
:106DC00037F000011650040AD8B433EF37F0E4EF7F
:106DD00037F00501476B486B496B4A6B05014B6BFC
:106DE0004C6B4D6B4E6B05014F6B506B516B526B87
:106DF0008BA0379BECEC22F000C1DAF101C1DBF192
:106E000002C1DCF103C1DDF100C13FF501C140F574
:106E100002C141F503C142F552EF37F00501476B5E
:106E2000486B496B4A6B05014B6B4C6B4D6B4E6B62
:106E300005014F6B506B516B526BECEC22F000C1B3
:106E4000DAF101C1DBF102C1DCF103C1DDF1E9ECF2
:106E500023F000C147F501C148F502C149F503C15E
:106E60004AF5E4EF37F0379BDAC13FF5DBC140F577
:106E7000DCC141F5DDC142F5ECEC22F000C14BF57F
:106E800001C14CF502C14DF503C14EF5E9EC23F00B
:106E900000C14FF501C150F502C151F503C152F5D2
:106EA00052EF37F0050161675DEF37F062675DEF24
:106EB00037F063675DEF37F0646761EF37F076EFC7
:106EC00037F0DAC100F1DBC101F1DCC102F1DDC153
:106ED00003F161C504F162C505F163C506F164C53E
:106EE00007F100EC30F003BFE4EF37F059C143F590
:106EF0005AC144F5B9C545F50501210E326F899A8D
:106F0000400EC76E200EC66E9E96C69E060EC96EB9
:106F1000FF0E9EB602D0E82EFCD7898A899A9E96EB
:106F2000C69E020EC96EFF0E9EB602D0E82EFCD79A
:106F30009E96C69E27C5C9FFFF0E9EB602D0E82EBC
:106F4000FCD79E96C69E26C5C9FFFF0E9EB602D0F0
:106F5000E82EFCD79E96C69E25C5C9FFFF0E9EB69D
:106F600002D0E82EFCD725EE37F0322F02D0C4EF46
:106F700037F09E96C69EDECFC9FFFF0E9EB602D0AA
:106F8000E82EFCD7B5EF37F0898A899A9E96C69E7F
:106F9000050EC96EFF0E9EB602D0E82EFCD79E9657
:106FA000C69EC952FF0E9EB602D0E82EFCD7C9B0CD
:106FB000CFEF37F0898A0501200E2527E86A2623BE
:106FC000E86A2723E86A282315900794120021C550
:106FD00000F122C501F123C502F124C503F1899A0C
:106FE000400EC76E200EC66E9E96C69E0B0EC96ED4
:106FF000FF0E9EB602D0E82EFCD79E96C69E02C11A
:10700000C9FFFF0E9EB602D0E82EFCD79E96C69E04
:1070100001C1C9FFFF0E9EB602D0E82EFCD79E9696
:10702000C69E00C1C9FFFF0E9EB602D0E82EFCD757
:107030009E96C69EC952FF0E9EB602D0E82EFCD781
:1070400025EE37F00501200E326F9E96C69EC9527E
:10705000FF0E9EB602D0E82EFCD7C9CFDEFF322F3E
:1070600025EF38F0898A1200899A400EC76E200EEB
:10707000C66E9E96C69E900EC96EFF0E9EB602D03C
:10708000E82EFCD79E96C69E000EC96EFF0E9EB6D9
:1070900002D0E82EFCD79E96C69E000EC96EFF0E4B
:1070A0009EB602D0E82EFCD79E96C69E000EC96EF4
:1070B000FF0E9EB602D0E82EFCD79E96C69EC95201
:1070C000FF0E9EB602D0E82EFCD7C9CF2DF59E96B6
:1070D000C69EC952FF0E9EB602D0E82EFCD7C9CF7D
:1070E0002EF5898A1200B6EC31F005012F51010A04
:1070F0005FE005012F51020A16E005012F51030A36
:1071000019E005012F51040A24E005012F51050A59
:107110002BE005012F51060A39E005012F51070A1E
:107120003FE0D8EF38F0602FD6EF38F05FC560F55C
:10713000D8EF38F0B0C500F101010F0E00170101C2
:107140000051000A35E001010051050A31E0D6EF97
:1071500038F0B0C500F101010F0E00170101005118
:10716000000A26E0D6EF38F00501B051000A20E011
:107170000501B051150A1CE00501B051300A18E0B4
:107180000501B051450A14E0D6EF38F00501B051C1
:10719000000A0EE00501B051300A0AE0D6EF38F0DF
:1071A0000501B051000A04E0D6EF38F01590120046
:1071B000158012008B90CCEC2EF0B9C5E8FFD708F3
:1071C00002E3CCEC2EF0B9C5E8FFC80802E3CCEC32
:1071D0002EF0B9C5E8FFB90802E3CCEC2EF0B9C532
:1071E000E8FFAA0802E3CCEC2EF0B9C5E8FF9B0843
:1071F00002E3CCEC2EF042EC36F0F29CF29E8B9443
:10720000C69AC2909482948C720ED36ED3A4FED789
:1072100089968A909390F29AF2949D909E909D9276
:107220009E92F298F2925CEC33F0FF0EE8CF00F001
:10723000E82EFED7002EFCD7F290F286815081A86E
:1072400024EF39F0F29E0300700ED36EF296F290A6
:0C72500015840380EDEC2EF09AEF0BF09B
:10BF0000E844F926000C160C2B0C3F0C520C640C68
:10BF1000760C860C960CA50CB30CC10CCF0CDC0C6B
:06BF2000E80CF40C000C1B
:0200000400F00A
:0100C800FE39
:00000001FF
